:100000000C9473000C949B000C949B000C949B002C
:100010000C949B000C9482090C949B000C949B0004
:100020000C949B000C949B000C949B000C949B00E4
:100030000C949B000C949B000C949B000C949B00D4
:100040000C940B1D0C949B000C94FC0C0C94D60C83
:100050000C949B000C949B000C949B000C949B00B4
:100060000C94B40D0C949B00BB13BD13BF13C113B0
:10007000C313C513C713C913FA13FD130014F713E1
:10008000031406141814181400000000240027009C
:100090002A0000000000250028002B0000000000BE
:1000A00023002600290004040404040404040202BA
:1000B00002020202030303030303010204081020E7
:1000C00040800102040810200102040810200000F2
:1000D0000008000201000003040700000000000007
:1000E00000001330E72F11241FBECFEFD8E0DEBF92
:1000F000CDBF26E0A0E8B4E001C01D92AB3EB20740
:10010000E1F714E0A0E0B1E0E0E2F0E702C0059022
:100110000D92A038B107D9F710E0C2E7D0E004C0D3
:100120002197FE010E945C34C137D107C9F70E94B4
:100130000F1F0C9403380C9400000F931F930E9420
:10014000FF1C009193041091940420919504309128
:100150009604DC01CB01801B910BA20BB30B853FF6
:100160009140A105B10508F4DEC161E080E00E9484
:10017000011E8FEB93E00E94251E6091E2047091B6
:10018000E3048091E4049091E50442E00E94871228
:1001900080E394E00E94251E80918A048130C1F49E
:1001A0000E94980F60E080E00E94011E8BEC93E0BB
:1001B0000E94251E809191049091920490930301D6
:1001C0008093020162E071E084E690E00E944F0FAC
:1001D00080918A048230D1F50E94980F60E080E01F
:1001E0000E94011E8DED93E00E94251E80919104D6
:1001F00090919204909349018093480120910201CB
:1002000030910301821B930B63E070E00E9407347E
:10021000260F371F3093010120930001260F371F4F
:10022000309347012093460160E071E087E690E05B
:100230000E944F0F66E471E08AE690E00E944F0F43
:1002400068E471E08DE690E00E944F0F80918A048F
:100250008330D1F50E94980F60E080E00E94011E7B
:100260008EEE93E00E94251E80919104909192045D
:1002700090934F0180934E012091480130914901A4
:10028000821B930B63E070E00E940734260F371F38
:1002900030934B0120934A01260F371F30934D01B5
:1002A00020934C016AE471E080E790E00E944F0FD8
:1002B0006CE471E083E790E00E944F0F6EE471E020
:1002C00086E790E00E944F0F80918A048430D1F538
:1002D0000E94980F60E080E00E94011E8FEF93E083
:1002E0000E94251E80919104909192049093550153
:1002F0008093540120914E0130914F01821B930B4A
:1003000063E070E00E940734260F371F30935101DD
:1003100020935001260F371F309353012093520131
:1003200060E571E089E790E00E944F0F62E571E0BF
:100330008CE790E00E944F0F64E571E08FE790E05A
:100340000E944F0F80918A04853009F048C00E94B6
:10035000980F60E080E00E94011E80E194E00E941E
:10036000251E809191049091920490935D01809359
:100370005C012091540130915501821B930B97FD34
:1003800003969595879595958795280F391F3093F6
:10039000570120935601280F391F3093590120939C
:1003A0005801820F931F90935B0180935A0166E579
:1003B00071E082E890E00E944F0F68E571E085E807
:1003C00090E00E944F0F6AE571E088E890E00E949B
:1003D0004F0F6CE571E08BE890E00E944F0F809129
:1003E0008A04863009F048C00E94980F60E080E0DF
:1003F0000E94011E81E294E00E94251E80919104DA
:1004000090919204909365018093640120915C0126
:1004100030915D01821B930B97FD0396959587950F
:1004200095958795280F391F30935F0120935E01C2
:10043000280F391F3093610120936001820F931FB1
:1004400090936301809362016EE571E08EE890E025
:100450000E944F0F60E671E081E990E00E944F0F2B
:1004600062E671E084E990E00E944F0F64E671E07B
:1004700087E990E00E944F0F80918A04873009F04D
:1004800048C00E94980F60E080E00E94011E82E355
:1004900094E00E94251E8091910490919204909383
:1004A0006D0180936C012091640130916501821B84
:1004B000930B97FD03969595879595958795280FAE
:1004C000391F3093670120936601280F391F30933D
:1004D000690120936801820F931F90936B018093B1
:1004E0006A0166E671E08AE990E00E944F0F68E6D3
:1004F00071E08DE990E00E944F0F6AE671E080EABA
:1005000090E00E944F0F6CE671E083EA90E00E9459
:100510004F0F0E94FF1C6093930470939404809388
:100520009504909396041F910F9108958F929F9236
:10053000AF92BF92FF920F931F93CF93DF93EC0183
:10054000F090A1040091A7041091A804F110A0C09C
:100550000230110509F49CC08130910509F04BC0AF
:1005600080918A048F5F873008F087E080938A0447
:1005700040914001509141016091420170914301CD
:100580008091830190918401A0918501B0918601B1
:10059000840F951FA61FB71F80938301909384013A
:1005A000A0938501B09386016091830170918401CD
:1005B0008091850190918601209140013091410107
:1005C000409142015091430180904001909041013F
:1005D000A0904201B09043010E941B34C501B401B8
:1005E0000E94F733609383017093840180938501A7
:1005F000909386014DC0019609F04AC04091400198
:1006000050914101609142017091430180918301B9
:1006100090918401A0918501B0918601841B950B76
:10062000A60BB70B8093830190938401A09385015F
:10063000B09386016091830170918401809185015E
:1006400090918601209140013091410140914201F9
:10065000509143018090400190904101A09042014F
:10066000B09043010E941B34C501B4010E94F733CE
:100670006093830170938401809385019093860138
:1006800080918A048150823008F481E080938A044A
:100690008091830190918401A0918501B0918601A0
:1006A000813C924CAA4DB64060F080EC92ECAAEDF1
:1006B000B6E08093830190938401A0938501B09369
:1006C00086018091830190918401A0918501B09170
:1006D0008601803A9648A140B10560F480EA96E828
:1006E000A1E0B0E08093830190938401A093850101
:1006F000B093860121E0F21249C0C130D10509F55D
:100700008091400190914101A0914201B09143013B
:1007100040918D0450918E0460918F0470919004EB
:10072000840F951FA61FB71F80938D0490938E048E
:10073000A0938F04B09390040130110509F07EC09E
:10074000B0C2CF3F8FEFD80709F5409140015091DB
:100750004101609142017091430180918D0490911B
:100760008E04A0918F04B0919004841B950BA60B6E
:10077000B70B80938D0490938E04A0938F04B09355
:1007800090040130110509F059C09CC201301105D7
:1007900009F054C08091A3049091A404A091A504F1
:1007A000B091A6048093830190938401A093850166
:1007B000B0938601C130D105C1F46EE671E08AE1E3
:1007C00090E00E94F60E40914001509141016091ED
:1007D000420170914301FC0180819181A281B3812A
:1007E000840F951FA61FB71F1BC0CF3FFFEFDF076A
:1007F00029F56EE671E08AE190E00E94F60E4091E4
:100800004001509141016091420170914301FC010E
:1008100080819181A281B381841B950BA60BB70BBC
:1008200080936E0190936F01A0937001B09371015A
:100830006EE671E08AE190E00E941C0F8091A704AF
:100840009091A804029709F073C0C130D10541F519
:100850008091A3049091A404A091A504B091A60452
:100860008093830190938401A0938501B0938601C6
:100870006BE974E085E190E00E94F60E4091400142
:10088000509141016091420170914301FC018081CE
:100890009181A281B381840F951FA61FB71F31C01C
:1008A000CF3FFFEFDF0709F043C08091A304909191
:1008B000A404A091A504B091A60480938301909311
:1008C0008401A0938501B09386016BE974E085E112
:1008D00090E00E94F60E40914001509141016091DC
:1008E000420170914301FC0180819181A281B38119
:1008F000841B950BA60BB70B181619061A061B06B8
:100900004CF480937E0190937F01A0938001B0937B
:10091000810108C010927E0110927F011092800127
:10092000109281016EE771E085E190E00E941C0F5A
:100930008091A7049091A804039709F040C080918A
:10094000A3049091A404A091A504B091A60480935F
:10095000830190938401A0938501B0938601C130F7
:10096000D10591F48093830190938401A093850134
:10097000B093860162E573E082E596E00E94800C08
:1009800081E08093820115C0CF3FFFEFDF0709F0C0
:100990005DC08093830190938401A0938501B093FF
:1009A00086016EE473E082E596E00E94800C10926E
:1009B000820162E871E08DE090E00E94760F809104
:1009C000A7049091A804049709F040C08091A30463
:1009D0009091A404A091A504B091A60480938301F2
:1009E00090938401A0938501B0938601C130D10515
:1009F00091F48093830190938401A0938501B09337
:100A0000860162E573E088E596E00E94800C81E053
:100A100080939F0415C0CF3F2FEFD20709F090C0FD
:100A20008093830190938401A0938501B093860104
:100A30006EE473E088E596E00E94800C10929F04BB
:100A40006FE974E080E090E00E94760F8091A70447
:100A50009091A804059709F073C0C130D10541F504
:100A60008091A3049091A404A091A504B091A60440
:100A70008093830190938401A0938501B0938601B4
:100A800066E771E088E290E00E94F60E4091400136
:100A9000509141016091420170914301FC018081BC
:100AA0009181A281B381840F951FA61FB71F31C00A
:100AB000CF3FFFEFDF0709F043C08091A30490917F
:100AC000A404A091A504B091A604809383019093FF
:100AD0008401A0938501B093860166E771E088E206
:100AE00090E00E94F60E40914001509141016091CA
:100AF000420170914301FC0180819181A281B38107
:100B0000841B950BA60BB70B181619061A061B06A5
:100B10004CF48093760190937701A0937801B09381
:100B2000790108C010927601109277011092780135
:100B30001092790166E771E088E290E00E941C0F54
:100B40008091A7049091A804069709F064C0C13071
:100B5000D10541F58091A3049091A404A091A5042E
:100B6000B091A6048093830190938401A0938501A2
:100B7000B093860167E974E084E290E00E94F60E8B
:100B800040914001509141016091420170914301B7
:100B9000FC0180819181A281B381840F951FA61FE2
:100BA000B71F2BC0CF3FFFEFDF07A9F58091A3044C
:100BB0009091A404A091A504B091A6048093830110
:100BC00090938401A0938501B093860167E974E056
:100BD00084E290E00E94F60E409140015091410164
:100BE0006091420170914301FC0180819181A28159
:100BF000B381841B950BA60BB70B8093970490933E
:100C00009804A0939904B0939A0467E974E084E28D
:100C100090E00E941C0F8091A7049091A804079770
:100C200079F5CF3FFFEFDF0799F48091A30490910E
:100C3000A404A091A504B091A6048093830190938D
:100C40008401A0938501B09386016EE473E014C023
:100C50002197B1F48091A3049091A404A091A504DC
:100C6000B091A6048093830190938401A0938501A1
:100C7000B093860162E573E08CE496E00E94800CFC
:100C80008091A7049091A804089769F5DF91CF910E
:100C90001F910F91FF90BF90AF909F908F900C94F9
:100CA0009D008091A3049091A404A091A504B0910B
:100CB000A6048093830190938401A0938501B0934F
:100CC00086017BCD8091A3049091A404A091A504FA
:100CD000B091A6048093830190938401A093850131
:100CE000B093860186CDDF91CF911F910F91FF9038
:100CF000BF90AF909F908F90089580918B049091BA
:100D00008C04009729F440E95AE36CE170E007C0D5
:100D100081309105A9F440ED51EB67E370E0409319
:100D20008301509384016093850170938601109232
:100D30008D0410928E0410928F041092900448C07B
:100D400082309105A9F440E153E96BE670E04093ED
:100D50008301509384016093850170938601109202
:100D60008D0410928E0410928F041092900438C05B
:100D700083309105A9F440E45BE66AE970E04093B2
:100D800083015093840160938501709386011092D2
:100D90008D0410928E0410928F041092900428C03B
:100DA00084309105A9F440E759EE67ED70E0409377
:100DB00083015093840160938501709386011092A2
:100DC0008D0410928E0410928F041092900420C013
:100DD0008530910529F480E49DE7A4E1B1E01EC0CF
:100DE0008630910529F480ED9FE3A4E4B1E016C0BC
:100DF0008730910529F480E99BE3AEE7B1E00EC0AE
:100E00008830910529F480E290EEA2EBB1E006C0B3
:100E10000997A1F480EC92E3AAE0B3E08093830108
:100E200090938401A0938501B093860110928D0464
:100E300010928E0410928F04109290040895809165
:100E400088049091890461E0019709F450C080E022
:100E50000E94011E8091400190914101A0914201A8
:100E6000B091430184369105A105B10589F188F45B
:100E70008A309105A105B10529F182339105A105BB
:100E8000B10519F10197A105B105C1F583E494E01D
:100E900033C0883E23E09207A105B105F9F030F494
:100EA000843F9140A105B105B1F00895803127E25A
:100EB0009207A105B105A9F0803A9648A140B10575
:100EC00099F0089588E494E017C08DE494E014C08C
:100ED00082E594E011C087E594E00EC08CE594E0D3
:100EE0000BC081E694E008C086E694E005C080E08F
:100EF0000E94011E8BE694E00C94251E08958091BB
:100F0000440190914501009739F421E030E030939D
:100F100089042093880444C08130910589F441E01C
:100F200050E060E070E040934001509341016093D5
:100F3000420170934301109289041092880430C0DA
:100F40008230910589F44AE050E060E070E040931F
:100F5000400150934101609342017093430110920C
:100F600089041092880424C08330910589F442E3F7
:100F700050E060E070E04093400150934101609385
:100F8000420170934301109289041092880418C0A2
:100F90008430910529F484E690E0A0E0B0E01EC022
:100FA0008530910529F484EF91E0A0E0B0E016C00F
:100FB0008630910529F488EE93E0A0E0B0E00EC001
:100FC0008730910529F480E197E2A0E0B0E006C007
:100FD000089781F480EA96E8A1E0B0E080934001B0
:100FE00090934101A0934201B09343011092890470
:100FF0001092880464E471E087E390E00C944F0F52
:10100000CF92DF92EF92FF9261E084E00E94011E96
:1010100060917E0170917F018091800190918101AA
:1010200020E432E44FE050E00E943D3469017A014F
:101030002093DE043093DF044093E0045093E104F6
:101040002A303105410551051CF480E20E944F1EF3
:10105000C701B6010E945D128EE20E944F1E609190
:101060007E0170917F01809180019091810120E447
:1010700032E44FE050E00E943D3428EE33E040E09F
:1010800050E00E943D3469017A012093DE043093E0
:10109000DF044093E0045093E10424363105410518
:1010A000510564F480E30E944F1E8AE0C816D10403
:1010B000E104F1041CF480E30E944F1EC701B60155
:1010C0000E945D128EE20E944F1E60917E0170911F
:1010D0007F01809180019091810128EE33E040E012
:1010E00050E00E943D346B017C016093DE047093FC
:1010F000DF048093E0049093E10484E6C816D104F1
:10110000E104F10464F480E30E944F1E8AE0C816F3
:10111000D104E104F1041CF480E30E944F1EC701D6
:10112000B6010E945D128AE494E0FF90EF90DF9098
:10113000CF900C94251ECF936DED74E088E090E085
:101140000E948E0FFC0180818093DD048091A004B9
:10115000811112C060E774E082E896E00E94800C82
:101160001092DD046DED74E088E090E00E94760F4F
:1011700060E080E10E94431CC091A004C13091F462
:101180006CE973E082E896E00E94800CC093DD0475
:101190006DED74E088E090E00E94760F61E080E100
:1011A0000E94431C8091A004823080F01092A00421
:1011B00060E774E082E896E00E94800C1092DD0403
:1011C0006DED74E088E090E00E94760F60EA74E0D4
:1011D00085E390E00E94760FCF910C94271ECF926A
:1011E000DF92EF92FF92CF93DF9360E083E00E9463
:1011F000011E80E20E944F1E609183017091840164
:10120000809185019091860120E432E44FE050E026
:101210000E941B3469017A012A30310518F480E2FA
:101220000E944F1E4AE0C701B6010E94581E8EE27E
:101230000E944F1E6091830170918401809185010D
:101240009091860120E432E44FE050E00E941B348C
:1012500028EE33E040E050E00E941B3469017A013F
:10126000E9012436310540F480E30E944F1E2A979D
:1012700018F480E30E944F1E4AE0C701B6010E94A5
:10128000581E8EE20E944F1E60918301709184016E
:10129000809185019091860128EE33E040E050E096
:1012A0000E941B346B017C01EB016436710540F434
:1012B00080E30E944F1E2A9718F480E30E944F1E7D
:1012C0004AE0C701B6010E94581E80E20E944F1EEC
:1012D00060E08FE00E94011E68E876E08FEC96E007
:1012E0000E94C80C60E080E00E94011E62E876E087
:1012F0008FEC96E0DF91CF91FF90EF90DF90CF9051
:101300000C94C80C1F920F920FB60F921124CF921B
:10131000DF92EF92FF920F931F932F933F934F9380
:101320005F936F937F938F939F93AF93BF93CF936D
:10133000DF93EF93FF93809190060E941A1CEC01BB
:1013400080918F060E941A1CE0918E06EF70CC0FE0
:10135000DD1F8C2B94E0E99FF0011124E357FE4F31
:10136000E80FF11DC081C0938E06C07359F10E9431
:10137000FF1C00918004109181042091820430911F
:1013800083046B017C01C01AD10AE20AF30AC092FD
:101390008404D0928504E0928604F09287046093DE
:1013A0008004709381048093820490938304C031FD
:1013B00019F481E090E004C0C03221F48FEF9FEF78
:1013C0000E949602FF91EF91DF91CF91BF91AF9173
:1013D0009F918F917F916F915F914F913F912F914D
:1013E0001F910F91FF90EF90DF90CF900F900FBE65
:1013F0000F901F901895FF920F931F93CF93DF9339
:10140000EC01F62E08811981C8010E947832F81685
:1014100021F06F2DC8010E948032CE01DF91CF9163
:101420001F910F91FF9008950895CF92DF92EF9250
:10143000FF920F931F93CF93DF936C017A018B017F
:10144000C0E0D0E0CE15DF0581F0D8016D918D01AF
:10145000D601ED91FC910190F081E02DC601099536
:10146000892B11F02196EECF7E01C701DF91CF913C
:101470001F910F91FF90EF90DF90CF900895FC01A6
:10148000538D448D252F30E0842F90E0821B930BE9
:10149000541710F0CF96089501970895FC01918D8F
:1014A000828D981761F0828DDF01A80FB11D5D96C6
:1014B0008C91928D9F5F9F73928F90E008958FEF34
:1014C0009FEF0895FC01918D828D981731F0828DE8
:1014D000E80FF11D858D90E008958FEF9FEF08953F
:1014E000FC01918D228D892F90E0805C9F4F821BA3
:1014F00091098F739927089583EA95E00E94700AF5
:1015000021E0892B09F420E0822F0895FC01848DCD
:10151000DF01A80FB11DA35ABF4F2C91848D90E01D
:1015200001968F739927848FA689B7892C93A089F8
:10153000B1898C91837080648C93938D848D981382
:1015400006C00288F389E02D80818F7D8083089515
:10155000EF92FF920F931F93CF93DF93EC0181E003
:10156000888F9B8D8C8D981305C0E889F9898081BF
:1015700085FD26C0F62E0B8D10E00F5F1F4F0F73F9
:101580001127E02E8C8DE8120CC00FB607FCFACFA5
:10159000E889F989808185FFF5CFCE010E94860A0E
:1015A000F1CF8B8DFE01E80FF11DE35AFF4FF08262
:1015B0009FB7F8940B8FEA89FB89808180620AC00B
:1015C0009FB7F894EE89FF896083E889F989808163
:1015D0008370806480839FBF81E090E0DF91CF9132
:1015E0001F910F91FF90EF900895CF93DF93EC013F
:1015F000888D8823C9F0EA89FB89808185FD05C033
:10160000A889B9898C9186FD0FC00FB607FCF5CF6C
:10161000808185FFF2CFA889B9898C9185FFEDCFB4
:10162000CE010E94860AE7CFDF91CF91089580E036
:1016300090E0892B29F00E947C0A81110C94000013
:10164000089585ED8093BC008091BC0084FDFCCFA3
:1016500010927E05089540910605262F30E0240F54
:10166000311D21323105DCF420917E052430C9F48E
:10167000FC0180E090E0861758F430910605219136
:10168000DC01AA51BB4FA30FB11D2C930196F3CFE0
:1016900080910605680F6093060580E0089581E05B
:1016A000089582E00895089508950895E0912E0523
:1016B00080912D05E81730F4F0E0E15DFA4F80816C
:1016C00090E008958FEF9FEF089590912E058091FF
:1016D0002D05981750F4E92FF0E0E15DFA4F2081D5
:1016E00030E09F5F90932E0502C02FEF3FEFC901BE
:1016F000089580912D0590E020912E05821B91097F
:101700000895CF92DF92EF92FF920F931F93CF93A2
:10171000DF937C01CB018A0120917F05222389F090
:10172000EB016B01C40ED51ECC15DD0569F0699186
:10173000D701ED91FC910190F081E02DC701099551
:10174000F3CF642F0E942B0BC801DF91CF911F9123
:101750000F91FF90EF90DF90CF900895CF93DF939C
:101760001F92CDB7DEB7698320917F052223D1F088
:101770002091A205203240F021E030E0FC013383CB
:10178000228380E090E015C080918005E82FF0E092
:10179000EF57FA4F998190838F5F809380058093F4
:1017A000A20505C061E0CE0101960E942B0B81E0ED
:1017B00090E00F90DF91CF91089580E090E0089540
:1017C0000E94E5370F931F93CF93DF93EC0188813D
:1017D0009981009729F02A813B812617370788F4E1
:1017E0008B016F5F7F4F0E941F37009761F09983D5
:1017F00088831B830A832C813D81232B11F4FC01F8
:10180000108281E001C080E0DF91CF911F910F91A4
:101810000895CF93DF93EC0160E08E810E94431C1A
:1018200061E08E810E94431C60E08E810E94431C17
:101830008BE891E00197F1F7DF91CF910895EF9256
:10184000FF920F931F93CF93DF936115710511F4EE
:1018500080E01CC041155105C1F07B01EC018C8179
:101860009D818A01080F191FB801CE010E94E20B69
:10187000882371F3288139818C819D81B701820F82
:10188000931F0E94FC371D830C8381E0DF91CF9171
:101890001F910F91FF90EF900895CF93DF93EC018C
:1018A00088819981009711F00E94963619821882DA
:1018B0001D821C821B821A82DF91CF910895EF92C4
:1018C000FF920F931F93CF93DF93EC017B018A016B
:1018D000BA010E94E20B811104C0CE010E944D0C9E
:1018E00007C01D830C83B701888199810E94FC3752
:1018F000CE01DF91CF911F910F91FF90EF9008954E
:10190000CF93DF93EC016115710559F0FB01019054
:101910000020E9F73197AF01461B570B0E945F0C7F
:1019200002C00E944D0CCE01DF91CF910895CF935C
:10193000DF93EC01FB018617970761F060817181ED
:101940006115710529F0448155810E945F0C02C028
:101950000E944D0CCE01DF91CF910895FC01808152
:1019600091810C949636FC011182108213821282AE
:10197000158214826115710551F0FB010190002060
:10198000E9F73197AF01461B570B0C945F0C089594
:10199000DB0114964D915C9115976D917C91DC0162
:1019A000ED91FC910280F381E02D09941F920F923A
:1019B0000FB60F9211242F933F934F935F936F9322
:1019C0007F938F939F93AF93BF93EF93FF9383EA9C
:1019D00095E00E94860AFF91EF91BF91AF919F9190
:1019E0008F917F916F915F914F913F912F910F90C8
:1019F0000FBE0F901F9018951F920F920FB60F9267
:101A000011242F938F939F93EF93FF93E091B3054E
:101A1000F091B4058081E091B905F091BA0582FD9D
:101A200012C090818091BC058F5F8F732091BD059E
:101A3000821751F0E091BC05F0E0ED55FA4F958F1B
:101A40008093BC0501C08081FF91EF919F918F91A0
:101A50002F910F900FBE0F901F901895CF92DF928D
:101A6000EF92FF920F931F93CF93DF936C017C0152
:101A700087E0E80EF11CC0E0D0E0062F10E0B801CE
:101A80000C2E02C0759567950A94E2F76170F70114
:101A900081917F010E94431C2196C430D10579F7C2
:101AA000C601DF91CF911F910F91FF90EF90DF90D2
:101AB000CF900C94090CCF92DF92EF92FF920F938C
:101AC0001F93CF93DF93EC01F62E642F8C810E943D
:101AD000431C8D818F3F19F060E00E94431C8F856D
:101AE0000F2D10E084FF25C06E0187E0C80ED11CC9
:101AF000E12CF12CB8010E2C02C0759567950A9463
:101B0000E2F76170F60181916F010E94431CFFEFC3
:101B1000EF1AFF0A88E0E816F10461F7CE01DF91C1
:101B2000CF911F910F91FF90EF90DF90CF900C9489
:101B3000090CB80184E0759567958A95E1F7CE01A7
:101B40000E942E0D6F2DCE01DF91CF911F910F912D
:101B5000FF90EF90DF90CF900C942E0D41E00E940B
:101B60005B0D81E090E008951F920F920FB60F92E7
:101B700011242F933F934F935F936F937F938F9392
:101B80009F93AF93BF93EF93FF938091B900887FAA
:101B9000803609F49CC068F5883209F45BC090F483
:101BA000803109F454C038F4882309F4F6C0883031
:101BB00009F44DC0F6C0883109F44CC0803209F4F4
:101BC0005DC0EFC0803409F468C048F4803309F484
:101BD00055C0883309F0E5C080937C05D8C08035B6
:101BE00009F44FC0883509F45DC0883409F0D9C0C4
:101BF000D6C0883909F4C7C0A8F4883709F467C08B
:101C000038F4883609F463C0803709F460C0C9C06D
:101C1000883809F4B8C0803909F45FC0803809F009
:101C2000C0C05BC0803B09F486C038F4803A09F438
:101C300066C0883A09F47FC0B4C0803C09F4A7C0EC
:101C4000883C09F4A4C0883B09F48AC0AAC08091EA
:101C5000590510C090917B0580917A05981770F511
:101C6000E0917B0581E08E0F80937B05F0E0E65AE2
:101C7000FA4F80818093BB0085EC86C080937C0501
:101C80008EC0E0917B0581E08E0F80937B05809173
:101C9000BB00F0E0E65AFA4F808390917B0580917B
:101CA0007A056EC0E0917B0581E08E0F80937B0505
:101CB0008091BB00F0E0E65AFA4F808380917D0569
:101CC00081116DC081E08093580584EA61C083E092
:101CD00080937E0510922805CFCF80912805803211
:101CE00008F051C0E091280581E08E0F809328050F
:101CF0008091BB00F0E0E85FFA4F8083BDCF85ECB8
:101D00008093BC0010927E0580912805803230F4CB
:101D1000E0912805F0E0E85FFA4F10826091280515
:101D200070E0E0912905F0912A0588E095E0099599
:101D30001092280536C084E080937E051092070536
:101D400010920605E0912B05F0912C0509958091E4
:101D50000605811105C081E0809306051092E60416
:101D6000E091070581E08E0F80930705F0E0EA51CE
:101D7000FB4F80818093BB00909107058091060501
:101D8000981708F479CF85E88093BC000AC085ECE9
:101D90008093BC0010927E0504C010927C050E94C6
:101DA000210BFF91EF91BF91AF919F918F917F9107
:101DB0006F915F914F913F912F910F900FBE0F90B8
:101DC0001F9018950F931F93CF93DF938C01EB0116
:101DD0000E9478328883C80101960E9478328983F4
:101DE000CE01DF91CF911F910F910895CF92DF9295
:101DF000EF92FF920F931F93CF93DF93EB017B0141
:101E000024E0E20EF11C8B016C01C61AD70AC60150
:101E1000800F911F0E947832F80181938F01EE1597
:101E2000FF05A9F7CE01DF91CF911F910F91FF9090
:101E3000EF90DF90CF900895AF92BF92CF92DF9254
:101E4000EF92FF920F931F93CF93DF9300D0CDB704
:101E5000DEB78B016B0124E0C20ED11C7B015C015B
:101E6000A61AB70AC5018E0D9F1DF70161917F016A
:101E70009A838983CE0101960E94FB09EC14FD042C
:101E800089F7C8010F900F90DF91CF911F910F91AB
:101E9000FF90EF90DF90CF90BF90AF900895EF92BA
:101EA000FF920F931F93CF93DF9300D0CDB7DEB790
:101EB0008C017B01FB0160819A838983CE010196AD
:101EC0000E94FB09F70161810F5F1F4F1A8309838D
:101ED000CE0101960E94FB09C7010F900F90DF9180
:101EE000CF911F910F91FF90EF9008950F931F9343
:101EF000CF93DF9300D0CDB7DEB78B01FB016081BC
:101F00009A838983CE0101960E94FB09C8010F9034
:101F10000F90DF91CF911F910F910895CF93DF9391
:101F2000EB010E9478328883CE01DF91CF91089532
:101F30008FE00E94AE1C9093920480939104BC01A8
:101F4000990F880B990B0E945B3120E030E040EA4A
:101F500050E40E94BA3120E030E040E85AE30E94A9
:101F6000BA316093E2047093E3048093E4049093A5
:101F7000E50408950F931F93CF93DF938B0191E0B6
:101F800090937F0590E69093A105109280051092A2
:101F9000A205682F80E496E00E94AE0BE801085F7E
:101FA0001F4F699180E496E00E94AE0BC017D107E5
:101FB000C1F781E0DF91CF911F910F910C94991E91
:101FC000CF93DF9391E090937F0590E69093A105E6
:101FD000109280051092A205682F80E496E00E947E
:101FE000AE0B81E00E94991E80917E058111FCCF8D
:101FF00081E080937E0510927D059FEF90937C0594
:1020000010927B0510927A058093590580915905AD
:10201000806C8093590580915805813061F410924D
:102020005805809159058093BB008091BC0083FDC9
:10203000F8CF85EC01C085EE8093BC0080917E05D1
:102040008130E1F380917B05811103C0C0917B0554
:1020500001C0C1E0EAE5F5E0AFE2B5E080E08C1751
:1020600021F091919D938F5FFACF10922E05C0932E
:102070002D0580912E05C81731F080E496E00E946E
:10208000650BD82FF6CF8D2FDF91CF910895CF9389
:10209000C0E1C80F8C2F0E94E00F682F63608C2F67
:1020A000CF910C94F51E1F93CF93DF93EC01162F65
:1020B00083E00E94E00F9E01332761E070E001C0E1
:1020C000660F2A95EAF7113019F46095682301C06C
:1020D000682B83E0DF91CF911F910C94F51E2F9216
:1020E0003F924F925F926F927F928F929F92AF92A8
:1020F000BF92CF92DF92EF92FF920F931F93CF93F5
:10210000DF93CDB7DEB761970FB6F894DEBF0FBE91
:10211000CDBF2D833E834F83588769877A871C0103
:102120001F870E876091CB067091CC068091CD06FB
:102130009091CE0624E630E040E050E00E94CA34A0
:102140002D87388B4B875C87762E672E582E492E2D
:102150008091C5069091C606A091C706B091C806A9
:102160006C017D01FF0CCC08DC2C76019C01AD01DB
:102170006C2D7C2D8C2D9C2D0FE10E949535A12C72
:102180000AECB02EEAE9CE2EFBE3DF2EE12CF12C97
:1021900000E010E00E94F734AD84B888CB84DC8482
:1021A000E72CF62C052D142D0E9462340FE10E94BD
:1021B000B03549015A01D501C401BB0F880B982FD6
:1021C000DC0189839A83AB83BC839401A501698177
:1021D000762F862F962FAD84B888CB84DC84E72CAD
:1021E000F62C052D0E94CC352983832E942E598BF5
:1021F000688B7B878C879D872D813E814F81588599
:1022000069857A85C1012F3FA7E53A07A7E44A0708
:10221000A8EF5A07ADE06A07710581059105A9F09D
:10222000A0F0211534404B46544F6441710581059F
:102230009105B9F0B0F01D8294E09E83ABE6AF83C8
:10224000B4EFB887E4E1E98709C01D82E8E5EE83D1
:10225000F7E4FF8328EF28878DE089871A86212CF1
:10226000312CA980B82CC92CD988E888FB840C852E
:102270001D852D813E814F81588569857A85C101F3
:102280000E94283529013A01FFE04F1651046104EC
:10229000710418F4AFE0AA2E08C02BE542165104D1
:1022A00061047104D0F0FAE5AF2EB12CC12CD12C11
:1022B000E12CF12C00E010E02981382D492D5989BD
:1022C00068897B858C859D850E9462342D833E8341
:1022D0004F83588769877A871C01A980B82CC92C3D
:1022E000D988E888FB840C851D852D813E814F812E
:1022F000588569857A85C1010E942635AA24AA9449
:10230000BB24BA94EFE0CE2ED12CE12CF12C00E0CE
:1023100010E00E946234A980B82CC92CD988E888C2
:10232000FB840C851D850E942835C901DA010097C0
:10233000A105B10529F4C12CD12C7601C39406C0A6
:10234000CC24CA94DC2C5FE0E52EF12CBC01CD013D
:1023500027E0660F771F881F991F2A95D1F737E06E
:10236000440C551C661C771C3A95D1F7A2E05A1A0A
:1023700061087108A70196010E941B34862E372E32
:10238000982E420E531E641E751E84E190E00E943A
:10239000FE359A838983FC01D082C182862D8370A9
:1023A000828353824482D701C6014CE0B695A7953B
:1023B000979587954A95D1F7807FC82EC90CC5821D
:1023C000368287828E859F85892B19F4BF018AE129
:1023D00007C0AE85BF85119729F469817A8182E2B1
:1023E0000E94BA0F89819A8161960FB6F894DEBF78
:1023F0000FBECDBFDF91CF911F910F91FF90EF9056
:10240000DF90CF90BF90AF909F908F907F906F9014
:102410005F904F903F902F900C94963610922E051F
:1024200010922D05109280051092A20510927E0543
:1024300081E080937D051092580561E082E10E9461
:10244000431C61E083E10E94431CE9EBF0E08081E2
:102450008E7F808380818D7F808388E48093B80025
:1024600085E48093BC0083E59BE090932C058093EA
:102470002B0584E59BE090932A0580932905089518
:102480000F931F93CF93DF938B01877028E0829F78
:10249000C001112480640E94551DE801085F1F4F90
:1024A00069918FEC96E00E94AE0DC017D107C1F77D
:1024B000DF91CF911F910F910895CF92DF92EF920C
:1024C000FF92CF93DF9397FF19C06B017C018DE2E0
:1024D0000E944F1EEC0166277727CB016C197D09FE
:1024E0008E099F094AE00E94581E8C0F9D1FDF91A4
:1024F000CF91FF90EF90DF90CF9008954AE0DF9169
:10250000CF91FF90EF90DF90CF900C94581E8F9258
:102510009F92AF92BF92CF92DF92EF92FF920F9372
:102520001F93CF93DF936B017C01142F9B01AC01B0
:102530000E94F233882319F084E794E027C0460113
:102540005701E894B7F82FEF3FEF4FE75FE7C5017A
:10255000B4010E94F23381110DC02FEF3FEF4FE71E
:102560005FE7C501B4010E94543118161CF488E7D6
:1025700094E00CC02FEF3FEF4FE75FE4C701B601D7
:102580000E94ED33181684F48CE794E0DF91CF912C
:102590001F910F91FF90EF90DF90CF90BF90AF9081
:1025A0009F908F900C94131E2FEF3FEF4FE75FEC3F
:1025B000C701B6010E94543187FDE6CF20E030E02C
:1025C000A901C701B6010E94543187FF09C08DE2FD
:1025D0000E944F1EEC01F7FAF094F7F8F09402C055
:1025E000C0E0D0E000E060E070E080E09FE3101722
:1025F00041F020E030E040E251E40E944C330F5FB4
:10260000F6CFA70196010E94E0326B017C010E9487
:10261000BE334B015C014AE00E94581EC80FD91F0F
:102620001123A9F1C501B4010E9459319B01AC01EC
:10263000C701B6010E94DF326B017C018EE20E946D
:102640004F1EC80FD91F20E030E040E251E4C7011F
:10265000B6010E94BA314B015C010E94BE336B018E
:10266000E12CF12C4AE0C701B6010E94581EC80FA8
:10267000D91FC701B6010E9459319B01AC01C501A8
:10268000B4010E94DF326B017C011150E1F6CE01F2
:10269000DF91CF911F910F91FF90EF90DF90CF903E
:1026A000BF90AF909F908F9008952F923F924F923E
:1026B0005F926F927F928F929F92AF92BF92CF92D2
:1026C000DF92EF92FF920F931F93CF93DF93CDB7DB
:1026D000DEB72E970FB6F894DEBF0FBECDBF3C011C
:1026E000C982DA82EB82FC820D831E832F833887B6
:1026F00049875A876B877C878BA18D873C2C2D2C33
:102700005E2C0E87412E922EC984DA84EB84FC84E1
:1027100084E190E00E94FE358C01FC01D082C182F0
:10272000862D880F880F880F845D0E94E00F952DFD
:1027300093708C7F892BF801828323823482D701A6
:10274000C6017CE0B695A795979587957A95D1F7C0
:10275000807F992D9F70C92EC80EC58246828E85B6
:10276000878398E069167104B8F4F301EC5CFF4FBD
:10277000B8010C945C348AE20DC082E30BC08AE39A
:1027800009C082E407C08AE405C082E503C08AE587
:1027900001C08BE50E94BA0F60E1F62EF60C8F2D7A
:1027A0000E94E00FE1E0682FAE1202C0606401C039
:1027B0006F7B8F2D0E94F51EF1E06F16710459F0AA
:1027C00038F092E06916710449F4A092C40618C06A
:1027D000A092C2060FC0A092C3060FC0E8E06E161A
:1027E0007104B0F4F301E45CFF4F0C945C3454E4E6
:1027F000B52E0EC04CE2B42E0BC034E3B32E08C08D
:102800002CE3B22E05C09CE4B92E02C084E5B82E9C
:102810008B2D0E94E00F8378FD85F1118C6090E193
:10282000899E40011124682F68298B2D0E94F51E76
:10283000C8012E960FB6F894DEBF0FBECDBFDF9154
:10284000CF911F910F91FF90EF90DF90CF90BF90AD
:10285000AF909F908F907F906F905F904F903F9040
:102860002F900C9496362F923F924F925F926F92D8
:102870007F928F929F92AF92BF92CF92DF92EF9210
:10288000FF920F931F93CF93DF93CDB7DEB7689777
:102890000FB6F894DEBF0FBECDBF522E3D87442E3B
:1028A0005E873B011C01A982B98ACA8ADB8AEC8A4D
:1028B000FD8A0E8B1F8B988A8F86211500EA3007C0
:1028C0000CEA400709EB500703E06007710581053A
:1028D000910511F008F046C02F3F10EE310715EFBB
:1028E000410715E05107610571058105910561F00A
:1028F00058F02F3F354D41415E47634071058105DA
:10290000910509F0D8F50BC0512CF1EEFD87B5EF1C
:102910004B2E05E00E87612C712C212C312C298146
:1029200039894A895B896C897D898E899F89A0E074
:102930000E94DE3509F0A7C0A52CBD84C42CDE841E
:102940007301810120E034E04BE654EF64E170E074
:1029500080E090E00E94283529873A874B875C8782
:10296000912C24C0512C10EA1D87FCEA4F2E29EB34
:102970002E87A3E06A2E712C212C312C29813989D4
:102980004A895B896C897D898E899F89A0E00E9434
:10299000DE3509F0F4C09924939414E0E12EF12C73
:1029A00000E010E0E986FA860B871C87E984FA8448
:1029B0000B851C85A801970160E070E0CB01A52C78
:1029C000BD84C42CDE847301810129833A834B8347
:1029D0005C836D837E838F83988760E070E080E006
:1029E00090E00E9462342983398B4A8B5B8B6C8B1D
:1029F0007D8B8E8B9F8BFF24F3949F1409F4C2C0B0
:102A000010E0812C912C5401839440E050E0BA01F5
:102A100001C011E0CB01BA0107E0660F771F881FE4
:102A2000991F0A95D1F7C984DA84EB84FC8427E0E6
:102A3000CC0CDD1CEE1CFF1C2A95D1F7A2E0DA1AA3
:102A4000E108F108A50194010E941B34C20ED31EB7
:102A5000E41EF51EEF85F889C082D182E282F382FE
:102A6000648375838683978380869186A286B386E6
:102A70001111BBC0298139894A895B896C897D899B
:102A80008E899F89B8C0188EA52CBD84C42CDE8485
:102A900073018101298139894A895B896C897D8922
:102AA0008E899F890E94283529873A874B875C87C2
:102AB00089859A85AB85BC850697A105B10520F46B
:102AC000B6E0AB2EB12C0FC0E984FA840B851C85CF
:102AD00029E0E21627E0F20601051105D0F0F8E042
:102AE000AF2EA7E0BA2EC12CD12CE12CF12C00E0A6
:102AF00010E0298139894A895B896C897D898E89B1
:102B00009F890E942835522E3D87442E5E873B01C7
:102B10001C01A52CBD84C42CDE8473018101298194
:102B200039894A895B896C897D898E899F890E9450
:102B30002635AA24AA94BB24BA94EFE0CE2ED12C39
:102B4000E12CF12C00E010E00E946234A52CBD8441
:102B5000C42CDE84730181010E942835A32FF42F39
:102B6000E52F422F5A2F6F2F7E2F411551056105FA
:102B70007105F9F4812C912C5401839420C081E0DB
:102B8000888F82CFAF85B8891D921D921D921C92AD
:102B90001397FD011482158216821782C12CD12C45
:102BA0007601C3941896CD92DD92ED92FC921B971C
:102BB00022C088248A94982C8FE0A82EB12CF88DFE
:102BC000F13009F026CFEF85F88910821182128248
:102BD0001382148215821682178281E090E0A0E0B1
:102BE000B0E080879187A287B387252D3D85442D4E
:102BF0005E85B301C10168960FB6F894DEBF0FBEC3
:102C0000CDBFDF91CF911F910F91FF90EF90DF909B
:102C1000CF90BF90AF909F908F907F906F905F907C
:102C20004F903F902F900895DF92EF92FF920F9375
:102C30001F93CF93DF93FC01E080F1800281138129
:102C4000D481C581B681D7809701A8016D2F7C2FD3
:102C50008B2F9D2D35534C40510961097109810914
:102C600091092F3F34434C405105610571058105A1
:102C7000910509F098F49701A8016D2F7C2F8B2FF7
:102C80009D2D07E00E949535208331834283538335
:102C9000648375838683978387E0FDC09701A801CD
:102CA0006D2F7C2F8B2F9D2D3A564841510961097C
:102CB0007109810991092F3F394648415105610544
:102CC00071058105910509F098F49701A8016D2F10
:102CD0007C2F8B2F9D2D06E00E949535208331831C
:102CE00042835383648375838683978386E0D3C04E
:102CF0009701A8016D2F7C2F8B2F9D2D345D4043B4
:102D0000510961097109810991092F3F334D4043F0
:102D10005105610571058105910509F098F4970148
:102D2000A8016D2F7C2F8B2F9D2D05E00E949535DE
:102D3000208331834283538364837583868397839F
:102D400085E0A9C09701A8016D2F7C2F8B2F9D2DA9
:102D5000385A4146510961097109810991092F3F8A
:102D6000374A41465105610571058105910509F014
:102D700098F49701A8016D2F7C2F8B2F9D2D04E0D7
:102D80000E94953520833183428353836483758306
:102D90008683978384E07FC09701A8016D2F7C2FE5
:102DA0008B2F9D2D3055434C5109610971098109C3
:102DB00091092F3F3F44434C510561057105810541
:102DC000910509F098F49701A8016D2F7C2F8B2FA6
:102DD0009D2D03E00E9495352083318342835383E8
:102DE000648375838683978383E055C09701A80128
:102DF0006D2F7C2F8B2F9D2D305A464851406109F5
:102E00007109810991092F3F3F49464851406105A9
:102E100071058105910509F098F49701A8016D2FBE
:102E20007C2F8B2F9D2D02E00E94953520833183CE
:102E300042835383648375838683978382E02BC0A8
:102E40009701A8016D2F7C2F8B2F9D2D30544D4065
:102E5000534061097109810991092F3F3F434D405A
:102E60005340610571058105910509F098F49701BA
:102E7000A8016D2F7C2F8B2F9D2D01E00E94953591
:102E8000208331834283538364837583868397834E
:102E900081E001C080E0DF91CF911F910F91FF9001
:102EA000EF90DF900895833081F028F4813099F01D
:102EB0008230A1F008958730A9F08830B9F08430CD
:102EC000D1F4809180008F7D03C0809180008F7746
:102ED00080938000089584B58F7702C084B58F7D7C
:102EE00084BD08958091B0008F7703C08091B000B9
:102EF0008F7D8093B00008953FB7F894809154057A
:102F000090915505A0915605B091570526B5A89BFF
:102F100005C02F3F19F00196A11DB11D3FBFBA2F6B
:102F2000A92F982F8827820F911DA11DB11DBC01CB
:102F3000CD0142E0660F771F881F991F4A95D1F790
:102F400008950F931F93CF938B01C0E1C80F8C2F6F
:102F50000E94E00F0115110511F48F7D04C00130AE
:102F6000110509F48062682F8C2FCF911F910F916A
:102F70000C94F51E2F923F924F925F926F927F9228
:102F80008F929F92AF92BF92CF92DF92EF92FF9279
:102F90000F931F93CF93DF93CDB7DEB7AA970FB6EA
:102FA000F894DEBF0FBECDBF622E298F732E3A8FED
:102FB0004B8F5C8F6D8F7E8F8F8F98A319A708A77B
:102FC00093012F3F34434C40510561057105810544
:102FD000910509F050F4198E85E38A8F8CE08B8F70
:102FE0001C8E1D8E1E8E1F8E18A2298D3A8D4B8D24
:102FF0005C8D6D8D7E8D8F8D98A12115304A4C4A48
:10300000594B634071058105910569F060F0198E97
:1030100080EA8A8F8CEA8B8F89EB8C8F83E08D8F8F
:103020001E8E1F8E18A2CE0149960E9414168AA7E2
:10303000798CBA8DAB8DFC8DED8D6E8C5F8C48A03C
:10304000272D3B2F4A2F5F2F6E2F762D852D942D08
:103050002F3F05ED300701E140070EE7500703E081
:10306000600771058105910511F008F07FC09E0190
:10307000235F3F4F4901A12CECE3BE2EF3E5CF2E99
:10308000ACE4DA2E10E1E12EF12C00E010E0272D67
:103090003B2F0E94331488A599A58130910509F42E
:1030A0004CC038F1029709F065C3898D8093BA0648
:1030B0008A8D8093BB068B8D8093BC068C8D80930C
:1030C000BD068D8D8093BE068E8D8093BF068F8D3D
:1030D0008093C00688A18093C10680E019A2212CAC
:1030E0003CE3332E43E5442E1CE41CA320E12DA336
:1030F0004CC3898D8093AA068A8D8093AB068B8DF5
:103100008093AC068C8D8093AD068D8D8093AE063A
:103110008E8D8093AF068F8D8093B00688A18093AB
:10312000B10680E019A2212C5CE3352E63E5462E22
:103130009CE49CA3E0E1EDA328C3898D8093B206B3
:103140008A8D8093B3068B8D8093B4068C8D80938B
:10315000B5068D8D8093B6068E8D8093B7068F8DC4
:103160008093B80688A18093B90604C3CE010D965A
:103170004C01A12CB12CC12CD12CE12CF12C00E064
:1031800010E0272D3B2F4A2F5F2F6E2F762D852D98
:10319000942D0E943314E8A5F9A5E130F10509F456
:1031A00058C020F0329709F49AC115C3298D3A8D81
:1031B0004B8D5C8D6D8D7E8D8E01035F1F4F4801A1
:1031C000A12CB12CC12CD12CE12CF12C00E010E071
:1031D0008F8D98A10E9433141901442E5CA36DA316
:1031E000772E582E692E60E070E080E090E00E941B
:1031F000A11720929A0630929B0640929C061CA131
:1032000010939D062DA120939E0670929F065092CA
:10321000A0066092A106898D8093AA068A8D80936C
:10322000AB068B8D8093AC068C8D8093AD068D8D17
:103230008093AE068E8D8093AF068F8D8093B006FF
:1032400088A18093B10681E031E039A31BA21AA2C4
:103250009FC21091CA06B98DAA8DFB8DEC8D0D8D84
:1032600009A30E8D0AA30F8D0EA308A10FA3123080
:1032700009F073C02B2F3A2F4F2F5E2F69A17AA12F
:103280008EA1902F30584A41564061097109810939
:1032900091092F37304E42475849624071058105E8
:1032A000910569F160F1A090BA06B090BB06C0909C
:1032B000BC06D090BD06E090BE06F090BF0600911F
:1032C000C0061091C1062B2F3A2F4F2F5E2F69A1F8
:1032D0007AA18EA19FA10E94D53589F01092B206E5
:1032E0001092B3061092B4061092B5061092B6066C
:1032F0001092B7061092B8061092B9066CC22090D0
:10330000A2063090A3064090A4062091A5062CA307
:103310003091A6063DA37090A7065090A806609035
:10332000A906CE010D964C015101C42CD22EE32EDC
:10333000F72C052D162D2B2F3A2F4F2F5E2F69A11D
:103340007AA18EA19FA10E94331461E070E081E018
:1033500090E00E94A11719A235C02093A2063093D5
:10336000A3064093A4065093A5066093A606709307
:10337000A7068093A8069093A9068E01035F1F4FAE
:103380004801A12CB12CC12CD12CE12CF12C00E056
:1033900010E02B2F3A2F4F2F5E2F69A17AA18EA11B
:1033A0009FA10E9433141901442E5CA36DA3772EB4
:1033B000582E692E61E070E081E090E00E94A11734
:1033C00011E019A3298D3A8D4B8D5C8D6D8D7E8D0D
:1033D0008F8D98A130584A41564061097109810981
:1033E00091092F37304E4247584962407105810597
:1033F000910509F008F457C081E08093CA06209136
:10340000BA063091BB064091BC065091BD06609152
:10341000BE067091BF068091C0069091C106A0E0E3
:103420000E94DE3509F442C08AEB96E00E94141631
:103430008AA7A090A206B090A306C090A406D09040
:10344000A506E090A606F090A7060091A8061091A8
:10345000A9062091BA063091BB064091BC06509156
:10346000BD066091BE067091BF06CE0101964C016B
:103470008091C0069091C1060E9433141F928AA4C5
:10348000A12CC980DA80EB80FC800D811E812F8108
:10349000388549855A856B857C8582E090E00E945D
:1034A00055130F9003C088E08093CA06898D8093DE
:1034B000B2068A8D8093B3068B8D8093B4068C8D73
:1034C0008093B5068D8D8093B6068E8D8093B7065A
:1034D0008F8D8093B80688A18093B90645C17090FE
:1034E000CA06B98DAA8DFB8DEC8D0D8D09A31E8D9D
:1034F0001AA30F8D0EA318A11FA301E0701273C0B1
:103500002B2F3A2F4F2F5E2F69A17AA18EA1912FD9
:1035100030584A41564061097109810991092F3794
:10352000304E42475849624071058105910569F165
:1035300060F1A090BA06B090BB06C090BC06D090D7
:10354000BD06E090BE06F090BF060091C006109147
:10355000C1062B2F3A2F4F2F5E2F69A17AA18EA182
:103560009FA10E94D53589F01092BA061092BB0631
:103570001092BC061092BD061092BE061092BF06B5
:103580001092C0061092C1062AC12090A206309067
:10359000A3064090A4062091A5062CA33091A60670
:1035A0003DA37090A7065090A8066090A906CE0192
:1035B0000D964C015101C42CD22EE32EF72C052D73
:1035C000162D2B2F3A2F4F2F5E2F69A17AA18EA196
:1035D0009FA10E94331461E070E082E090E00E94BD
:1035E000A11719A235C02093A2063093A3064093D9
:1035F000A4065093A5066093A6067093A706809331
:10360000A8069093A9068E01035F1F4F4801A12CC5
:10361000B12CC12CD12CE12CF12C00E010E02B2F8F
:103620003A2F4F2F5E2F69A17AA18EA19FA10E94F0
:1036300033141901442E5CA36DA3772E582E692EE6
:1036400061E070E082E090E00E94A11711E019A310
:10365000298D3A8D4B8D5C8D6D8D7E8D8F8D98A1D2
:1036600030584A41564061097109810991092F3743
:10367000304E42475849624071058105910509F075
:1036800008F457C082E08093CA062091B2063091B8
:10369000B3064091B4065091B5066091B60670919C
:1036A000B7068091B8069091B906A0E00E94DE3579
:1036B00009F442C082EB96E00E9414168AA7A090FB
:1036C000A206B090A306C090A406D090A506E090F4
:1036D000A606F090A7060091A8061091A9062091D1
:1036E000B2063091B3064091B4065091B506609190
:1036F000B6067091B706CE0101964C018091B806CE
:103700009091B9060E9433141F928AA4A12CC980FB
:10371000DA80EB80FC800D811E812F813885498500
:103720005A856B857C8581E090E00E9455130F904F
:1037300003C088E08093CA06898D8093BA068A8D7B
:103740008093BB068B8D8093BC068C8D8093BD06C9
:103750008D8D8093BE068E8D8093BF068F8D809356
:10376000C00688A18093C10681E0E1E0F0E0FBA300
:10377000EAA30EC080E019A2212C9CE3392E23E598
:10378000422EFCE4FCA300E10DA3712C512C612C12
:103790008F938AA4A82ECD84DE84EF84F8880989CB
:1037A0001A892B893C894D895E896F89788D88A516
:1037B00099A50E9455130F9019A1113079F40AA10F
:1037C0001BA19101442D5CA16DA1772D852D962D16
:1037D0000E946F1003C07724739401C0712C872D51
:1037E000AA960FB6F894DEBF0FBECDBFDF91CF9182
:1037F0001F910F91FF90EF90DF90CF90BF90AF900F
:103800009F908F907F906F905F904F903F902F9000
:103810000895009769F0FC0101900020E9F73197C5
:10382000AF01481B590BBC018AE696E00C941F0CB3
:1038300080E00895CF93DF93282F30E0F901E25321
:10384000FF4F8491F901E654FF4FD491F901EA55F5
:10385000FF4FC491CC2391F081110E945317EC2F9C
:10386000F0E0EE0FFF1FE456FF4FA591B491EC91ED
:10387000ED2381E090E021F480E002C080E090E060
:10388000DF91CF9108951F93CF93DF93282F30E0DE
:10389000F901E253FF4F8491F901E654FF4FD491AF
:1038A000F901EA55FF4FC491CC23C1F0162F8111C5
:1038B0000E945317EC2FF0E0EE0FFF1FEE56FF4F64
:1038C000A591B4919FB7F894111104C08C91D09533
:1038D000D82302C0EC91DE2BDC939FBFDF91CF9108
:1038E0001F910895CF93DF9390E0FC01E654FF4FC2
:1038F0002491FC01EA55FF4F8491882361F190E007
:10390000880F991FFC01E857FF4FC591D491FC0126
:10391000EE56FF4FA591B491611109C09FB7F8947D
:103920008881209582238883EC912E230BC06230FE
:1039300061F49FB7F8948881322F30958323888370
:10394000EC912E2B2C939FBF06C08FB7F894E88183
:103950002E2B28838FBFDF91CF9108958E3008F0F2
:103960008E508770806480937C0080917A008064A0
:1039700080937A0080917A0086FDFCCF8091780058
:103980002091790090E0922B08958F929F92AF92B0
:10399000BF92CF92DF92EF92FF926B017C010E9467
:1039A0007C174B015C01C114D104E104F104F1F076
:1039B0000E947C17DC01CB0188199909AA09BB096F
:1039C000883E9340A105B10570F321E0C21AD108E9
:1039D000E108F10888EE880E83E0981EA11CB11C56
:1039E000C114D104E104F10419F7DDCFFF90EF9089
:1039F000DF90CF90BF90AF909F908F9008952FB79A
:103A0000F894609150057091510580915205909104
:103A100053052FBF08951F920F920FB60F921124D6
:103A20002F933F938F939F93AF93BF9380915005B4
:103A300090915105A0915205B091530530914F05D9
:103A400023E0230F2D3720F40196A11DB11D05C0E1
:103A500026E8230F0296A11DB11D20934F058093E8
:103A6000500590935105A0935205B0935305809152
:103A7000540590915505A0915605B09157050196B2
:103A8000A11DB11D8093540590935505A093560533
:103A9000B0935705BF91AF919F918F913F912F9117
:103AA0000F900FBE0F901F90189540E0682F8FEC7D
:103AB00096E00C945B0DCF93DF93823028F09091C9
:103AC000DE0698609093DE068093E2061092E3068D
:103AD00080E48093E40680E18093E50680E58093AE
:103AE000E60661E08091D3060E94721C8091D406A4
:103AF0008F3F19F061E00E94721C61E08091D50651
:103B00000E94721CCFECD6E09E012F5C3640809163
:103B1000DE0684FD03C084E090E002C088E090E00F
:103B20002196281739072CF461E08E810E94721CBF
:103B3000EBCF8BE39DE00197F1F760E08091D30636
:103B40000E94431C60E08091D5060E94431C809136
:103B5000D4068F3F19F060E00E94431C8091DE067E
:103B600084FD20C063E08FEC96E00E942E0DCBE434
:103B7000D6E4CE010197F1F763E08FEC96E00E9466
:103B80002E0D2197F1F763E08FEC96E00E942E0D49
:103B900083E592E00197F1F762E08FEC96E00E94F6
:103BA0002E0D15C080620E94551D8BE496E401978E
:103BB000F1F78091DE0680620E94551D83E592E058
:103BC0000197F1F78091DE0680620E94551D809179
:103BD000DE0680620E94551D84E08093DF068CE043
:103BE0000E94551D81E00E94551D8BE39FE10197C6
:103BF000F1F782E08093E00686E0DF91CF910C94AC
:103C0000551D643008F063E09091E206691710F0EA
:103C10006FEF690FE62FF0E0E153F94F9489890FB8
:103C200080680C94551D009769F0FC0101900020FC
:103C3000E9F73197AF01481B590BBC018FEC96E0B7
:103C40000C94150A80E090E008950C94131EEF92F6
:103C5000FF920F931F93CF93DF9300D0CDB7DEB7C2
:103C600082E8E82E86E0F82E0EE210E0F70161917E
:103C70007F011A830983CE0101960E94FB090F5F21
:103C80001F4F0433110591F782E896E00F900F90D3
:103C9000DF91CF911F910F91FF90EF90089541E038
:103CA000682F8FEC96E00E945B0D81E090E0089514
:103CB0008F929F92AF92BF920F931F93CF93DF93F8
:103CC000CDB7DEB7A1970FB6F894DEBF0FBECDBF5C
:103CD00019A2423008F44AE08E010F5D1F4F842E76
:103CE000912CA12CB12CA50194010E941B34E62F2C
:103CF000B901CA0101501109EA3014F4E05D01C0B4
:103D0000E95CD801EC93232B242B252B61F7C80108
:103D10000E94131EA1960FB6F894DEBF0FBECDBF52
:103D2000DF91CF911F910F91BF90AF909F908F9097
:103D30000895282F3091A205313208F04AC08091B1
:103D40007E058111FCCF9091A10542E040937E0554
:103D500020937D052FEF20937C0510927B053093F7
:103D60007A05E1E8F5E0AAE5B5E020E0321721F0B8
:103D700041914D932F5FFACF10925905209159052B
:103D8000990F922B9093590590915805913061F4B9
:103D900010925805909159059093BB009091BC00EA
:103DA00093FDF8CF95EC01C095EE9093BC009091F7
:103DB0007E059230E1F390917C059F3F79F08091F0
:103DC0007C05803241F080917C05803331F084E0C5
:103DD00005C081E003C082E001C083E0109280054D
:103DE0001092A20510927F050895CF93C62F91E0FF
:103DF00090937F0590E69093A10510928005109214
:103E0000A205682F80E496E00E94AE0B6C2F80E440
:103E100096E00E94AE0B81E0CF910C94991ECF9357
:103E2000DF93CDB7DEB7AB970FB6F894DEBF0FBE0A
:103E3000CDBF789484B5826084BD84B5816084BD33
:103E400085B5826085BD85B5816085BD80916E0038
:103E5000816080936E001092810080918100826069
:103E600080938100809181008160809381008091A6
:103E700080008160809380008091B1008460809395
:103E8000B1008091B00081608093B00080917A0091
:103E9000846080937A0080917A00826080937A00B7
:103EA00080917A00816080937A0080917A008068A6
:103EB00080937A001092C100E091B305F091B405AF
:103EC00082E08083E091AF05F091B0051082E0912F
:103ED000B105F091B2058FEC80831092BB05E091A3
:103EE000B705F091B80586E08083E091B505F091C3
:103EF000B605808180618083E091B505F091B605BB
:103F0000808188608083E091B505F091B60580815D
:103F100080688083E091B505F091B60580818F7D42
:103F2000808382E00E945B1D81E00E94551D8BE32F
:103F30009FE10197F1F70E940E1261E08AE00E9472
:103F4000721C61E08BE00E94721C61E08CE00E94B8
:103F5000721C61E08DE00E94721C60E08FE00E94A4
:103F6000721C61E080E10E94721C61E081E10E94AC
:103F7000721C64E371E081E00E9440126CE271E027
:103F800082E00E94401264E271E083E00E944012ED
:103F90006CE171E084E00E94401264E171E085E030
:103FA0000E9440126CE071E086E00E94401264E0E2
:103FB00071E087E00E94401269EA74E089E090E0D5
:103FC0000E948E0FDC018C91823F09F0B0C38EE01D
:103FD0000E94AE1C853F91403CF08EE00E94AE1CDA
:103FE0008A3892400CF4A3C36FE974E080E090E05B
:103FF0000E948E0FDC018C9180939F0462E871E037
:104000008DE090E00E948E0FFC0180818093820100
:104010006BE974E085E190E00E94F60EFC0180817E
:104020009181A281B38180937E0190937F01A093BF
:104030008001B09381016EE671E08AE190E00E9418
:10404000F60EFC0180819181A281B38180936E0183
:1040500090936F01A0937001B09371016CE371E0D4
:104060008FE190E00E94F60EFC0180819181A28197
:10407000B3818093830190938401A0938501B093D1
:10408000860167E974E084E290E00E94F60EFC018C
:1040900080819181A281B381809372019093730199
:1040A000A0937401B093750166E771E088E290E037
:1040B0000E94F60EFC0180819181A281B3818093E0
:1040C000760190937701A0937801B093790192E8FB
:1040D000A92E96E0B92E0EE210E0C8010E947832B7
:1040E000D5018D935D010F5F1F4F04331105A9F7B3
:1040F00062E876E0CB010E94970C60EA74E085E309
:1041000090E00E948E0FFC0180818093A00464E403
:1041100071E087E390E00E94E20EDC018D919C91BA
:10412000909345018093440180916E0190916F01BD
:10413000A0917001B09171018093C5069093C6065D
:10414000A093C706B093C8060E940E1262E987EBDF
:104150000E94F51E8FE00E94E00F40EC5CEF6BE9DF
:1041600071E04093CB065093CC066093CD067093DC
:10417000CE06682F6F738FE00E94F51E60E880E125
:104180000E94F51E60E881E10E94F51E60E882E170
:104190000E94F51E6CE080E10E94F51E6CE081E15A
:1041A0000E94F51E6CE082E10E94F51E60E281EB48
:1041B0000E94F51E60E881EB0E94F51E00E010E011
:1041C00020E03CE343E55CE460E170E080E090E007
:1041D0000E946F1061E081E090E00E94531080E047
:1041E00090E00E94471081E090E00E94471082E03A
:1041F00090E00E94471069ED71E088E896E00E9427
:10420000800C62E08EE00E94721C809168008460E5
:104210008093680080916D008C6080936D0078942D
:104220000E94FF1C60938004709381048093820439
:104230009093830488EE93E0A0E0B0E08093840440
:1042400090938504A0938604B09387040E94EF089E
:1042500088EEC82E83E0D82EE12CF12C3324339441
:104260006CE371E08FE190E00E94F60EFC0180812A
:104270009181A281B38180933C0190933D01A093F1
:104280003E01B0933F0140918301509184016091C0
:1042900085017091860180913C0190913D01A09132
:1042A0003E01B0913F01481759076A077B0731F07B
:1042B00063E871E08FE190E00E941C0F8091880418
:1042C00090918904019709F093C0809184049091A2
:1042D0008504A0918604B091870485369105A105D7
:1042E000B105C0F02AE030E040E050E0209340010A
:1042F0003093410140934201509343018EE690E098
:10430000A0E0B0E08093840490938504A093860499
:10431000B09387048091840490918504A0918604D1
:10432000B09187048997A109B109CC97A105B1057E
:10433000C0F422E330E040E050E0209340013093AD
:104340004101409342015093430186E490E0A0E094
:10435000B0E08093840490938504A0938604B09386
:1043600087048091840490918504A0918604B09183
:1043700087044F97A109B1090A97A105B105C0F4B7
:1043800024E630E040E050E02093400130934101CA
:10439000409342015093430183E290E0A0E0B0E0FB
:1043A0008093840490938504A0938604B09387043B
:1043B0008091840490918504A0918604B091870433
:1043C0004F97A105B105A0F4C0924001D0924101E0
:1043D000E0924201F09243012FE030E040E050E0F3
:1043E000209384043093850440938604509387047B
:1043F0008091A7049091A804892B11F40E94EF08E2
:104400008EE00E94AE1C8EE00E94AE1C5C01909378
:10441000AD048093AC046AE070E080E090E00E941C
:10442000C51C8EE00E94AE1C8EE00E94AE1C092EC0
:10443000000CAA0BBB0BA5010B2C000C660B770B19
:104440002C013D0133E0431A5108610871084415FD
:1044500055056605770564F00396A11DB11D841707
:104460009507A607B70724F0B092B704A092B60448
:10447000A090B604B090B70445E8A41643E0B40693
:104480006CF01092AB048091AA0481112FC160E0FE
:1044900081E10E94431C1092DC0428C158E4A51657
:1044A000B10464F48091AB04811108C061E081E142
:1044B0000E94431C3092DC043092AB04C501895445
:1044C00091098D34910530F58091AB04811122C0A2
:1044D0008091AA0481110AC061E081E10E94431C1D
:1044E0003092AA043092DC043092AB048091AB0489
:1044F0008111FCC01091AA04113009F0F7C060E0EE
:1045000081E10E94431C1092AA041092DC041093D3
:10451000AB04ECC0C501875991098034910500F5C1
:104520008091AB0481111CC08091A104811108C04D
:104530003092A1043092AB041092B5041092B404EE
:104540008091AB0481110CC08091A104813041F4B1
:104550001092A1048093AB041092B5041092B4049D
:10456000C501885D9109C697A8F48091AB048111BB
:1045700011C080918B0490918C0401968A30910532
:10458000DCF010928C0410928B043092AB040E94E9
:104590007D06ACC0C5018F509140C19790F48091C9
:1045A000AB0481110EC080918B0490918C04019713
:1045B00097FF02C089E090E090938C0480938B0475
:1045C000E4CFC501815491408C9700F58091AB04F4
:1045D00081111CC08091C204811104C03092C204B8
:1045E0003092AB048091AB04811108C08091C20469
:1045F000813021F41092C2048093AB048091A00416
:104600008F5F8093A0040E949B0870C0C5018E56E6
:1046100091408297D0F48091AB04811116C08091B3
:10462000D204811104C03092D2043092AB04809144
:10463000AB0481115BC08091D204813009F056C077
:104640001092D2048093AB0451C0C50181599140AE
:104650008297A8F48091AB04811111C0809144012C
:1046600090914501019689309105E4F01092450141
:10467000109244013092AB040E947F0737C0C501FD
:104680008F5A91408336910590F48091AB0481114B
:104690000EC08091440190914501019797FF02C09F
:1046A00088E090E09093450180934401E3CF83E15B
:1046B000A81A82E0B80A97E7A916B104B8F4809165
:1046C000AB04811113C08091A7049091A8040196B6
:1046D0009093A8048093A70430928A04099724F049
:1046E0001092A8041092A7043092AB048091DC04CD
:1046F0008093CB048091830190918401A0918501E6
:10470000B091860180349244AF40B10508F4DDC019
:104710008091830190918401A0918501B0918601DF
:10472000803C964CAD42B10508F4F3C0CEC06FE9B1
:1047300074E080E090E00E94760F82EF90E09A8330
:104740008983BE016F5F7F4F89E090E00E944F0F29
:1047500062E871E08DE090E00E94760F67EC74E013
:104760008FE090E00E941C0F6EE771E085E190E021
:104770000E941C0F6EE671E08AE190E00E941C0F1F
:1047800063E871E08FE190E00E941C0F62E771E046
:1047900084E290E00E941C0F66E771E088E290E0FE
:1047A0000E941C0F0E94271E60EA74E085E390E0DF
:1047B0000E94760F64E471E087E390E00E944F0F5F
:1047C00062E071E084E690E00E944F0F60E071E0EB
:1047D00087E690E00E944F0F66E471E08AE690E081
:1047E0000E944F0F68E471E08DE690E00E944F0F49
:1047F0006AE471E080E790E00E944F0F6CE471E0A2
:1048000083E790E00E944F0F6EE471E086E790E04E
:104810000E944F0F60E571E089E790E00E944F0F22
:1048200062E571E08CE790E00E944F0F64E571E073
:104830008FE790E00E944F0F66E571E082E890E01C
:104840000E944F0F68E571E085E890E00E944F0FED
:104850006AE571E088E890E00E944F0F6CE571E036
:104860008BE890E00E944F0F6EE571E08EE890E0DB
:104870000E944F0F60E671E081E990E00E944F0FC7
:1048800062E671E084E990E00E944F0F64E671E017
:1048900087E990E00E944F0F66E671E08AE990E0B8
:1048A0000E944F0F68E671E08DE990E00E944F0F83
:1048B0006AE671E080EA90E00E944F0F6CE671E0DA
:1048C00083EA90E00E944F0F8FCB809183019091FB
:1048D0008401A0918501B0918601803C964CAD4247
:1048E000B10510F40C94AF2E809183019091840156
:1048F000A0918501B091860180349B44AC44B10500
:1049000010F00C94AF2E84E085B981E090E00C9417
:10491000AA2F15B810928C0410928B048091A704D2
:104920009091A804009781F04091830150918401F7
:1049300060918501709186014093A3045093A40473
:104940006093A5047093A6042091DC04213009F043
:10495000CCC0892B09F0C9C0A090AE04B090AF04C0
:1049600085010F5F1F4F1093AF040093AE0484E1E5
:104970000E94AE1CBC01990F880B990B0E945B3101
:104980004B015C0185E10E94AE1CBC01990F880BB4
:10499000990B0E945B312B013C019B01AC01C501CD
:1049A000B4010E94ED3387FD07C061E080E00E9402
:1049B000011E8BED91E097C0043111050CF495C0F8
:1049C0001092AF041092AE04A3019201C501B4018C
:1049D0000E94E03268A779A78AA79BA7A501940146
:1049E000C301B2010E94DF329B01AC0168A579A529
:1049F0008AA59BA50E944C334B015C0120E030E06E
:104A0000A9010E94ED33181624F0B7FAB094B7F854
:104A1000B09420E030E040EA50E4C301B2010E94CB
:104A2000BA3120E030EC4FE754E40E944C332CE2E2
:104A300038E540EB5CE30E944C339B01AC010E94E3
:104A4000BA3120E030E048E452E40E944C332B01BC
:104A50003C0120E030E040E050E4C501B4010E9498
:104A6000E03268A779A78AA79BA7A501940160E017
:104A700070E080E89FE30E944C339B01AC0168A585
:104A800079A58AA59BA50E94E0329B01AC0160E05C
:104A900070E080E890E40E944C33A30192010E94F0
:104AA000BA312B013C0161E080E00E94011E8EEED4
:104AB00091E00E94251E42E0C501B4010E948712C8
:104AC00061E088E00E94011E83EF91E00E94251EB4
:104AD00061E08BE00E94011E40E0C301B2010E9430
:104AE000871287EF91E00E94251E91E08091A1043A
:104AF000813009F090E081E02091DC04211180E018
:104B0000892309F419C18091A7049091A804892BE5
:104B100009F012C180917A0190917B01A0917C01F2
:104B2000B0917D01803A56E8950751E0A507B1059F
:104B3000A4F48091830190918401A0918501B091AA
:104B40008601805A9648A140B109B095A0959095EC
:104B500081959F4FAF4FBF4F17C0813C924CAA4DDC
:104B6000B640D4F08091830190918401A091850199
:104B7000B091860120EC32EC4AED56E0281B390B4F
:104B80004A0B5B0BDA01C90180938D0490938E046C
:104B9000A0938F04B09390048091B6049091B704D1
:104BA00087599109C197D0F48091B4049091B504CC
:104BB000843691059CF401969093B5048093B404D7
:104BC000C29761F410928D0410928E0410928F049B
:104BD000109290041092B5041092B4040E941F0722
:104BE0008090830190908401A0908501B09086010F
:104BF00080918D0490918E04A0918F04B0919004C7
:104C0000880E991EAA1EBB1E80927A0190927B018B
:104C1000A0927C01B0927D0161E084E00E94011EBF
:104C200080E20E944F1EC501B40120E432E44FE04F
:104C300050E00E943D3449015A012093B004309362
:104C4000B1044093B2045093B3043AE08316910444
:104C5000A104B1041CF480E20E944F1EC501B401FE
:104C60000E945D128EE20E944F1E60917A01709147
:104C70007B0180917C0190917D0120E432E44FE042
:104C800050E00E943D34A70196010E943D34490145
:104C90005A012093B0043093B1044093B20450936E
:104CA000B30444E684169104A104B10464F480E3DF
:104CB0000E944F1E5AE085169104A104B1041CF411
:104CC00080E30E944F1EC501B4010E945D128EE276
:104CD0000E944F1E60917A0170917B0180917C014E
:104CE00090917D01A70196010E943D344B015C012A
:104CF0006093B0047093B1048093B2049093B304B2
:104D000084E688169104A104B10464F480E30E944F
:104D10004F1E9AE089169104A104B1041CF480E3AB
:104D20000E944F1EC501B4010E945D1280E20E94E4
:104D30004F1E80E20E944F1E91E08091DC048111A1
:104D400090E081E02091A104211180E0892309F401
:104D500026C28091A7049091A804892B09F01FC254
:104D600064EA72E08AE696E00E94800C0E94980F46
:104D70000E94FF1C0E94FF1C80909304909094045A
:104D8000A0909504B0909604DC01CB018819990994
:104D9000AA09BB0984369105A105B10510F40C944C
:104DA000B02F0E94FF1CDC01CB0188199909AA09C8
:104DB000BB0984369105A105B10578F00E94FF1C5E
:104DC000DC01CB0188199909AA09BB09883C910526
:104DD000A105B10510F40C94BA2F0E94FF1CDC0150
:104DE000CB0188199909AA09BB09883C9105A1053D
:104DF000B10578F00E94FF1CDC01CB0188199909EC
:104E0000AA09BB098C329140A105B10510F40C949C
:104E1000C42F0E94FF1CDC01CB0188199909AA0943
:104E2000BB098C329140A105B10578F00E94FF1CAE
:104E3000DC01CB0188199909AA09BB098039914085
:104E4000A105B10510F40C94CE2F0E94FF1CDC01CB
:104E5000CB0188199909AA09BB0980399140A1059C
:104E6000B10578F00E94FF1CDC01CB01881999097B
:104E7000AA09BB09853F9140A105B10510F40C9426
:104E8000D82F0E94FF1CDC01CB0188199909AA09BF
:104E9000BB09853F9140A105B10508F47EC1209171
:104EA000C0043091C1048091BE049091BF04820F70
:104EB000931F2091BC043091BD04820F931F209159
:104EC000BA043091BB04820F931F2091B804309133
:104ED000B904820F931F65E070E00E9407345B0104
:104EE00070939204609391046CE671E083EA90E021
:104EF0000E94E20EDC018D919C91A816B9061CF06F
:104F00008CEF91E034C16CE671E083EA90E00E949E
:104F1000E20EFC01808191818A159B051CF489E0D9
:104F200092E025C16AE671E080EA90E00E94E20E1C
:104F3000DC018D919C918A159B051CF486E192E021
:104F400016C168E671E08DE990E00E94E20EFC0176
:104F5000808191818A159B051CF483E292E007C150
:104F600066E671E08AE990E00E94E20EDC018D9134
:104F70009C918A159B051CF480E392E0F8C064E6DE
:104F800071E087E990E00E94E20EFC01808191814E
:104F90008A159B051CF48DE392E0E9C062E671E09E
:104FA00084E990E00E94E20EDC018D919C918A15CB
:104FB0009B051CF48AE492E0DAC060E671E081E9C6
:104FC00090E00E94E20EFC01808191818A159B0590
:104FD0001CF487E592E0CBC06EE571E08EE890E0CE
:104FE0000E94E20EDC018D919C918A159B051CF4B8
:104FF00084E692E0BCC06CE571E08BE890E00E9432
:10500000E20EFC01808191818A159B051CF481E7E9
:1050100092E0ADC06AE571E088E890E00E94E20E9F
:10502000DC018D919C918A159B051CF48EE792E022
:105030009EC068E571E085E890E00E94E20EFC0108
:10504000808191818A159B051CF48BE892E08FC0CA
:1050500066E571E082E890E00E94E20EDC018D914D
:105060009C918A159B051CF488E992E080C064E558
:1050700071E08FE790E00E94E20EFC018081918157
:105080008A159B051CF485EA92E071C062E571E027
:105090008CE790E00E94E20EDC018D919C918A15D4
:1050A0009B051CF482EB92E062C060E571E089E749
:1050B00090E00E94E20EFC01808191818A159B059F
:1050C0001CF48FEB92E053C06EE471E086E790E051
:1050D0000E94E20EDC018D919C918A159B051CF4C7
:1050E0008CEC92E044C06CE471E083E790E00E94B5
:1050F000E20EFC01808191818A159B051CF489EDEB
:1051000092E035C06AE471E080E790E00E94E20E30
:10511000DC018D919C918A159B051CF486EE92E032
:1051200026C068E471E08DE690E00E94E20EFC018A
:10513000808191818A159B051CF483EF92E017C052
:1051400066E471E08AE690E00E94E20EDC018D9157
:105150009C918A159B051CF480E093E008C066E4EE
:1051600071E087E690E00E94E20E8DE093E00E94FD
:10517000091C61E084E00E94011E6AE676E08FEC83
:1051800096E00E94C80C0E94FF1C609393047093E9
:10519000940480939504909396040E941F07809135
:1051A000A7049091A804181619060CF03AC10197AB
:1051B00001F560E080E00E94011E8AE193E00E9418
:1051C000251E0E941F0761E084E00E94011E82EA02
:1051D00092E00E94251E60916E0170916F01809196
:1051E0007001909171010E945D1281ED92E00E9428
:1051F000251E8091A7049091A804029761F40E9453
:10520000000860E080E00E94011E8CE293E00E94B2
:10521000251E0E941F078091A7049091A804039760
:1052200059F50E94000860E080E00E94011E8DE3B5
:1052300093E00E94251E80918201811106C06EE4D8
:1052400073E082E596E00E94800C809182018130BB
:1052500031F462E573E082E596E00E94800C61E043
:1052600080E00E94011E62E576E08FEC96E00E94ED
:10527000C80C80E20E944F1E8091A7049091A80460
:10528000049771F560E080E00E94011E86E593E0DE
:105290000E94251E80919F04811106C06EE473E078
:1052A00088E596E00E94800C80919F04813031F463
:1052B00062E573E088E596E00E94800C61E080E0A2
:1052C0000E94011E81EA92E00E94251E68E576E0B8
:1052D0008FEC96E00E94C80C88E693E00E94251EA1
:1052E0008091A7049091A804059719F560E080E0EB
:1052F0000E94011E86E793E00E94251E0E941F0760
:1053000061E084E00E94011E82EA92E00E94251E74
:105310006091760170917701809178019091790187
:105320000E945D1287E893E00E94251E80E20E94A1
:105330004F1E8091A7049091A804069701F560E0A4
:1053400080E00E94011E8FE893E00E94251E0E94CB
:105350001F0761E084E00E94011E82EA92E00E9441
:10536000251E609197047091980480919904909102
:105370009A040E945D1287E893E00E94251E8091A6
:10538000A7049091A8040797F1F460E080E00E94E0
:10539000011E80EA93E00E94251E82EA92E00E94AC
:1053A000251E61E080E00E94011E85EC92E00E94D3
:1053B000251E6CE476E08FEC96E00E94C80C89EB29
:1053C00092E00E94251E8091A7049091A80408975E
:1053D00041F58091500690915106892B11F1009171
:1053E0004C0610914D066EE473E0C8010E94F3373D
:1053F000892B21F41092A8041092A70462E573E0AF
:10540000C8010E94F337892B11F40E949D008091FE
:10541000A7049091A804099724F01092A804109270
:10542000A7049091DB048091A004981731F00E94AA
:105430009B088091A0048093DB040E947F078091E9
:10544000C7049091C804A091C904B091CA04809384
:10545000C3049093C404A093C504B093C6046BE93D
:1054600074E085E190E00E94F60EFC01808191815C
:10547000A281B38180937E0190937F01A0938001EC
:10548000B09381011091DC04113081F4809183018B
:1054900090918401A0918501B091860180937A0159
:1054A00090937B01A0937C01B0937D014091830197
:1054B0005091840160918501709186018091D204A0
:1054C00040385F49654D710508F485C0811178C089
:1054D00069ED71E088E896E00E94800C60EB73E073
:1054E00086E796E00E94800C8091A104813029F526
:1054F000409076015090770160907801709079012A
:1055000040917E0150917F016091800170918101F5
:1055100080907A0190907B01A0907C01B0907D01F9
:10552000840C951CA61CB71C8091C7049091C804DC
:10553000A091C904B091CA0426C081114EC18091C6
:10554000830190918401A0918501B09186014090E2
:1055500076015090770160907801709079014091C8
:105560007E0150917F016091800170918101809056
:10557000C7049090C804A090C904B090CA04840CD9
:10558000951CA61CB71C880D991DAA1DBB1D840F58
:10559000951FA61FB71F8093D7049093D804A0939C
:1055A000D904B093DA04440D551D661D771D409350
:1055B0007E0150937F0160938001709381010DC142
:1055C000813049F464EB73E088E896E00E94800C37
:1055D00066EB73E018C040918301509184016091A3
:1055E00085017091860140385F49654D710508F06D
:1055F00016C1811174C064EB73E088E896E00E94E4
:10560000800C60EB73E086E796E00E94800C80914E
:10561000A1048130E9F440917A0150917B016091BD
:105620007C0170917D018091C7049091C804A09184
:10563000C904B091CA04840F951FA61FB71F4091DB
:105640007E0150917F0160918001709181011EC0A7
:10565000811128C08091830190918401A0918501DE
:10566000B09186018090C7049090C804A090C904AE
:10567000B090CA0440917E0150917F0160918001F9
:1056800070918101480D591D6A1D7B1D840F951F66
:10569000A61FB71F8093D7049093D804A093D90472
:1056A000B093DA048091C204813009F0B8C011309F
:1056B00009F0B5C04091D7045091D8046091D90445
:1056C0007091DA048091720190917301A09174013C
:1056D000B0917501840F951FA61FB71F98C0813028
:1056E00009F09DC069ED71E088E896E00E94800CA9
:1056F00066EB73E086E796E00E94800C8091A1043F
:10570000813069F540907601509077016090780182
:105710007090790140917E0150917F0160918001EC
:105720007091810180917A0190917B01A0917C011F
:10573000B0917D01840D951DA61DB71D840F951F89
:10574000A61FB71F8090C7049090C804A090C904FA
:10575000B090CA04880D991DAA1DBB1D1CCF8111D4
:105760003CC08090830190908401A0908501B0900E
:105770008601409176015091770160917801709196
:10578000790180917E0190917F01A0918001B0917B
:105790008101840F951FA61FB71F880E991EAA1E90
:1057A000BB1E4091C7045091C8046091C904709118
:1057B000CA04480D591D6A1D7B1D4093D7045093A0
:1057C000D8046093D9047093DA0480937E01909397
:1057D0007F01A0938001B09381018091C204813048
:1057E000F1F41130E1F48091D7049091D804A091A4
:1057F000D904B091DA044091720150917301609123
:10580000740170917501841B950BA60BB70B8093E7
:10581000D7049093D804A093D904B093DA0480916C
:105820007A0190917B01A0917C01B0917D01209142
:10583000D20480383FE9930735EDA307B105C8F1DD
:1058400021111AC02091A104213009F0CCC040914F
:10585000C7045091C8046091C9047091CA04840FB0
:10586000951FA61FB71F40917E0150917F01609147
:1058700080017091810189C0213009F0B4C020916C
:10588000A104213009F0AFC04091C7045091C80471
:105890006091C9047091CA04840F951FA61FB71F99
:1058A00040917E0150917F01609180017091810152
:1058B0001BC0211142C02091A104213009F093C0E6
:1058C00040917E0150917F01609180017091810132
:1058D000840F951FA61FB71F4091C7045091C8049D
:1058E0006091C9047091CA04840F951FA61FB71F49
:1058F0008093D7049093D804A093D904B093DA048A
:105900008091C204813009F06EC0113009F06BC083
:105910004091D7045091D8046091D9047091DA0471
:105920008091720190917301A0917401B091750101
:10593000840F951FA61FB71F4EC0213009F053C01A
:105940002091A104213009F04EC040917E01509178
:105950007F016091800170918101840F951FA61FC6
:10596000B71F4091C7045091C8046091C904709159
:10597000CA04840F951FA61FB71F4091760150914E
:1059800077016091780170917901840F951FA61FAE
:10599000B71F8093D7049093D804A093D904B093F1
:1059A000DA048091C2048130F1F41130E1F4809185
:1059B000D7049091D804A091D904B091DA04409111
:1059C0007201509173016091740170917501841B93
:1059D000950BA60BB70B8093D7049093D804A09394
:1059E000D904B093DA0480919F04813029F461E0F6
:1059F00081E090E00E94531080919F04811105C0C6
:105A000060E081E090E00E9453108091820181115A
:105A100005C060E082E090E00E9453108091820116
:105A2000813029F461E082E090E00E9453104091BF
:105A3000D7045091D8046091D9047091DA04809110
:105A4000D3049091D404A091D504B091D604481702
:105A500059076A077B0709F053C0209186063091E9
:105A6000870680918006909181062817390709F0F2
:105A700047C0809182069091830660917C06709168
:105A80007D06009719F061157105A1F46115710586
:105A900049F0232B99F0DB018C9190E09195819551
:105AA00091090AC0009751F0232B41F0FC0180813D
:105AB00090E002C00E94F337892B11F59091D20437
:105AC0008091D10498131CC09091A1048091D004BE
:105AD000981316C040917E0150917F016091800122
:105AE000709181018091CC049091CD04A091CE045D
:105AF000B091CF04481759076A077B0709F42BC1F7
:105B00006091D7047091D8048091D9049091DA04FF
:105B100024E630E040E050E00E94CA3400E010E0AB
:105B20000E94BA1760918301709184018091850170
:105B30009091860124E630E040E050E00E94CA34B3
:105B400001E010E00E94BA1760917E0170917F0120
:105B5000809180019091810124E630E040E050E0A6
:105B60000E94BB3402E010E00E94BA178091A104A9
:105B70008093D0048091D7049091D804A091D90447
:105B8000B091DA048093D3049093D404A093D50405
:105B9000B093D60462E876E08CE796E00E94970C1A
:105BA0008091D2048093D1048091CB048093DC0453
:105BB00080917E0190917F01A0918001B09181013F
:105BC0008093CC049093CD04A093CE04B093CF04E3
:105BD000609183017091840180918501909186018B
:105BE0001BA21AA21DA21CA21FA21EA22AE0AE0185
:105BF0004F5F5F4F0E940831BE016F5F7F4FCE0144
:105C000082960E94800C80915E0690915F060097BC
:105C1000C9F06AA17BA16115710591F04091600600
:105C2000509161062EA13FA14217530748F00E94F0
:105C3000FC378EA19FA1909363068093620618C0E3
:105C40000E9496368AA19BA190935F0680935E0680
:105C50008CA19DA190936106809360068EA19FA167
:105C600090936306809362061BA21AA21DA21CA237
:105C70001FA21EA2CE0182960E94AE0C80916206E7
:105C8000909163060B9798F51BA21AA21DA21CA265
:105C90001FA21EA24AE0BE016F5F7F4F80E090E02E
:105CA0000E94FD30BE016F5F7F4FCE0182960E9441
:105CB000800C409162065091630660915E0670917F
:105CC0005F06CE0182960E941F0C811104C0CE0196
:105CD00082960E944D0CBE016E5D7F4F8EE596E070
:105CE0000E94970CCE0182960E94AE0CC7CF6AEB41
:105CF00073E0CE0101960E94B30C40916206509170
:105D0000630660915E0670915F06CE0101960E9467
:105D10001F0C811104C0CE0101960E944D0C41E080
:105D200050E06DEB73E0CE0101960E941F0C8823BA
:105D300009F448C1BE016F5F7F4F83EA95E00E947E
:105D4000C80CCE0101960E94AE0C64E170E080E0C8
:105D500090E00E94C51C0E94170B0C94302180918A
:105D6000830190918401A0918501B09186018034D6
:105D70009B44AC44B10590F08091830190918401E3
:105D8000A0918501B091860181159241AA47B10584
:105D900028F488E085B982E090E0DCC0809183013E
:105DA00090918401A0918501B09186018115924165
:105DB000AA47B10590F08091830190918401A09150
:105DC0008501B091860181159B41A74BB10528F44F
:105DD0008CE085B983E090E0BDC080918301909113
:105DE0008401A0918501B091860181159B41A74B4B
:105DF000B10590F08091830190918401A09185017B
:105E0000B091860181159442A44FB10528F480E138
:105E100085B984E090E09EC08091830190918401D7
:105E2000A0918501B091860181159442A44FB105DE
:105E300090F08091830190918401A0918501B091AF
:105E40008601803C9A4EA142B14028F484E185B994
:105E500085E090E07FC08091830190918401A091C2
:105E60008501B0918601803C9A4EA142B14090F0EC
:105E70008091830190918401A0918501B091860168
:105E80008038914BAF44B14028F488E185B986E071
:105E900090E060C08091830190918401A091850180
:105EA000B09186018038914BAF44B14068F0809149
:105EB000830190918401A0918501B0918601803C7D
:105EC0009C4FAB49B140F8F08091830190918401DF
:105ED000A0918501B0918601803C9C4FAB49B140B7
:105EE000B8F08091830190918401A0918501B091D7
:105EF000860181159A45A246B24050F480E285B9E8
:105F000088E090E027C08CE185B987E090E022C06E
:105F10008091830190918401A0918501B0918601C7
:105F200081159A45A246B24010F40C948E248091BB
:105F3000830190918401A0918501B0918601813CFB
:105F40009B43A744B34010F00C948E2484E285B99F
:105F500089E090E090938C0480938B040C948E24C1
:105F600080919104909192049093C1048093C00415
:105F70000C94D12680919104909192049093BF0447
:105F80008093BE040C94ED2680919104909192042C
:105F90009093BD048093BC040C94092780919104D4
:105FA000909192049093BB048093BA040C9425279B
:105FB00080919104909192049093B9048093B804D5
:105FC0000C944127CE0101960E944D0CB3CE8CE477
:105FD00096E00E94AE0C82E596E00E94AE0C88E549
:105FE00096E00E94AE0C8EE596E00E94AE0C84E630
:105FF00096E00E94AE0C8AE696E00E94AE0C80E726
:1060000096E00E94AE0C86E796E00E94AE0C8CE70C
:1060100096E00E94AE0C82E896E00E94AE0C88E802
:1060200096E00C94AE0CCF93DF93E3EAF5E0138295
:10603000128288EE93E0A0E0B0E084839583A6838B
:10604000B7832DEA31E03183208325EC30E03587BA
:10605000248724EC30E03787268720EC30E0318B32
:10606000208B21EC30E0338B228B22EC30E0358B1F
:10607000248B26EC30E0378B268B118E128E138EFC
:10608000148EE0E4F6E01382128284839583A68363
:10609000B7838FEB91E091838083EFECF6E013827E
:1060A000128281ED91E09183808389E084838FEF78
:1060B0008583C8E0C68387E0878386E0808785E0A4
:1060C000818784E082871386148615861686178654
:1060D00081E00E945B1DE1E9F6E0C0AFC1AF11AA0B
:1060E00012AA13AA1186128613861486158616869E
:1060F0001786108A118A128A138A148A158A168AB8
:10610000178A108E118E128E138E148E158E168E87
:10611000178E10A211A212A213A214A215A216A2E7
:1061200017A210A611A612A613A614A615A616A6A7
:1061300017A610AA80EC9CEFABE9B1E082AF93AF59
:10614000A4AFB5AFCEE8D6E083E0898382E08A834E
:1061500060E083E00E94721C60E08A810E94721CF1
:1061600061E089810E94431C61E08A810E94431C96
:10617000188269ED71E088E896E00E94B30C60E750
:1061800074E082E896E00E94B30C60E774E08CE76C
:1061900096E00E94B30C60EB73E086E796E00E9405
:1061A000B30C64EA72E080E796E00E94B30C64EA04
:1061B00072E08AE696E00E94B30C64EA72E084E63C
:1061C00096E00E94B30C64EA72E08EE596E00E94CD
:1061D000B30C6EE473E088E596E00E94B30C62E5D0
:1061E00073E082E596E00E94B30C6EE473E08CE409
:1061F00096E0DF91CF910C94B30CBB274A3031F479
:10620000992322F4BDE2909581959F4F0C942B31F8
:10621000BB27FA01A62F6217710581059105330B83
:1062200030FB66F0AA27660F771F881F991FAA1FE9
:10623000A21710F0A21B63953850A9F7A05DAA33EE
:1062400008F0A95DA19336F7B111B1931082CA018C
:106250000C944431BB27FB015527AA27880F991FAF
:10626000AA1FA41710F0A41B83955051B9F7A05D85
:10627000AA3308F0A95DA193009779F7B111B19302
:106280001192CB010C944431DC01FC01672F719118
:106290007723E1F7329704C07C916D93708362910C
:1062A000AE17BF07C8F308950E94963108F481E045
:1062B0000895E89409C097FB3EF4909580957095F9
:1062C00061957F4F8F4F9F4F9923A9F0F92F96E942
:1062D000BB279395F695879577956795B795F111B7
:1062E000F8CFFAF4BB0F11F460FF1BC06F5F7F4F54
:1062F0008F4F9F4F16C0882311F096E911C0772366
:1063000021F09EE8872F762F05C0662371F096E86E
:10631000862F70E060E02AF09A95660F771F881F3D
:10632000DAF7880F9695879597F90895990F0008E1
:10633000550FAA0BE0E8FEEF16161706E807F90757
:10634000C0F012161306E407F50798F0621B730BF2
:10635000840B950B39F40A2661F0232B242B252B73
:1063600021F408950A2609F4A140A6958FEF811D16
:10637000811D08950E94CD310C943E320E9430322E
:1063800038F00E94373220F0952311F00C94273218
:106390000C942D3211240C9472320E944F3270F3FF
:1063A000959FC1F3950F50E0551F629FF001729FBA
:1063B000BB27F00DB11D639FAA27F00DB11DAA1FC9
:1063C000649F6627B00DA11D661F829F2227B00D16
:1063D000A11D621F739FB00DA11D621F839FA00DA1
:1063E000611D221F749F3327A00D611D231F849FF1
:1063F000600D211D822F762F6A2F11249F57504048
:106400009AF0F1F088234AF0EE0FFF1FBB1F661FC2
:10641000771F881F91505040A9F79E3F510580F08B
:106420000C9427320C9472325F3FE4F3983ED4F31D
:10643000869577956795B795F795E7959F5FC1F72F
:10644000FE2B880F911D9695879597F9089597F9DA
:106450009F6780E870E060E008959FEF80EC08950A
:1064600000240A9416161706180609060895002433
:106470000A9412161306140605060895092E0394AD
:10648000000C11F4882352F0BB0F40F4BF2B11F421
:1064900060FF04C06F5F7F4F8F4F9F4F089557FD80
:1064A0009058440F551F59F05F3F71F04795880F82
:1064B00097FB991F61F09F3F79F087950895121619
:1064C00013061406551FF2CF4695F1DF08C01616C5
:1064D00017061806991FF1CF869571056105089476
:1064E0000895E894BB2766277727CB0197F908958D
:1064F000F999FECF92BD81BDF89A992780B508958C
:10650000262FF999FECF1FBA92BD81BD20BD0FB6CF
:10651000F894FA9AF99A0FBE019608950E94D03223
:10652000A59F900DB49F900DA49F800D911D1124E7
:1065300008952F923F924F925F926F927F928F9227
:106540009F92AF92BF92CF92DF92EF92FF920F9302
:106550001F93CF93DF93CDB7DEB7CA1BDB0B0FB60C
:10656000F894DEBF0FBECDBF09942A8839884888C9
:106570005F846E847D848C849B84AA84B984C8845F
:10658000DF80EE80FD800C811B81AA81B981CE0F56
:10659000D11D0FB6F894DEBF0FBECDBFED0108953B
:1065A000A29FB001B39FC001A39F700D811D112454
:1065B000911DB29F700D811D1124911D0895505899
:1065C000BB27AA270E94F7320C943E320E94303239
:1065D00038F00E94373220F039F49F3F19F426F446
:1065E0000C942D320EF4E095E7FB0C942732E92F42
:1065F0000E944F3258F3BA17620773078407950752
:1066000020F079F4A6F50C9471320EF4E0950B2E7F
:10661000BA2FA02D0B01B90190010C01CA01A001F4
:106620001124FF27591B99F0593F50F4503E68F14F
:106630001A16F040A22F232F342F4427585FF3CF90
:10664000469537952795A795F0405395C9F77EF461
:106650001F16BA0B620B730B840BBAF09150A1F0AA
:10666000FF0FBB1F661F771F881FC2F70EC0BA0F30
:10667000621F731F841F48F4879577956795B795B8
:10668000F7959E3F08F0B0CF9395880F08F09927B3
:10669000EE0F9795879508950E9460330C943E32D3
:1066A0000E94373258F00E94303240F029F45F3FA8
:1066B00029F00C94273251110C9472320C942D3223
:1066C0000E944F3268F39923B1F3552391F3951B40
:1066D000550BBB27AA2762177307840738F09F5F03
:1066E0005F4F220F331F441FAA1FA9F335D00E2E70
:1066F0003AF0E0E832D091505040E695001CCAF7DD
:106700002BD0FE2F29D0660F771F881FBB1F26179F
:1067100037074807AB07B0E809F0BB0B802DBF0176
:10672000FF2793585F4F3AF09E3F510578F00C9445
:1067300027320C9472325F3FE4F3983ED4F386958F
:1067400077956795B795F7959F5FC9F7880F911D66
:106750009695879597F90895E1E0660F771F881F52
:10676000BB1F621773078407BA0720F0621B730B05
:10677000840BBA0BEE1F88F7E09508950E945732FC
:1067800088F09F5798F0B92F9927B751B0F0E1F0F2
:10679000660F771F881F991F1AF0BA95C9F714C0A2
:1067A000B13091F00E947132B1E008950C947132D1
:1067B000672F782F8827B85F39F0B93FCCF38695DB
:1067C00077956795B395D9F73EF490958095709538
:1067D00061957F4F8F4F9F4F08950E94963108F427
:1067E0008FEF08950E949631880B990B0895DB0175
:1067F0008F939F930E948E32BF91AF91A29F800D85
:10680000911DA39F900DB29F900D1124089597FBA9
:10681000072E16F4009407D077FD09D00E94EA35C0
:1068200007FC05D03EF4909581959F4F0895709593
:1068300061957F4F0895A1E21A2EAA1BBB1BFD0193
:106840000DC0AA1FBB1FEE1FFF1FA217B307E4074F
:10685000F50720F0A21BB30BE40BF50B661F771FA7
:10686000881F991F1A9469F7609570958095909587
:106870009B01AC01BD01CF010895052E97FB1EF4CD
:1068800000940E94543457FD07D00E941B3407FC2B
:1068900003D04EF40C945434509540953095219586
:1068A0003F4F4F4F5F4F089590958095709561953C
:1068B0007F4F8F4F9F4F0895EE0FFF1F0590F4916C
:1068C000E02D0994DF93CF931F930F939A9DF02DA2
:1068D000219FF00D8B9DF00D8A9DE02DF10D039F02
:1068E000F00D029FE00DF11D4E9DE00DF11D5E9D2E
:1068F000F00D4F9DF00D7F936F93BF92AF925F931A
:106900004F93D5010E94D0328B01AC01D7010E9478
:10691000D032EB01E80FF91FD6010E94B2342F915B
:106920003F91D6010E94D032C60FD71FE81FF91F32
:10693000AF91BF910E94B2342F913F910E94D0320B
:10694000C60FD71FE81FF91FD6010E94D032E60FED
:10695000F71F9801BE01CF0111240F911F91CF9114
:10696000DF9108950E94D032460F571FC81FD91FCC
:1069700008F43196089597FB57FF0C94CB349F93FE
:106980008F930E94CB346E1B7F0BAF91BF918A0B0C
:106990009B0B0895E894DF93CF93FC01DB010E94E9
:1069A000D0327F936F93E9019A01AC01BF93AF930B
:1069B0003F932F93DF010E94D03226F46C1B7D0B96
:1069C000820B930B9E01EB01FC010E94B234AF914C
:1069D000BF912F913F910E94B234BE01CF01F901C6
:1069E0002F913F91CF91DF910895689401C0E89471
:1069F000F92FF12B12F00C942935A0E0B0E0E3E080
:106A0000F5E30C949F32092E059422F40E948535FB
:106A1000112392F4F0E80F26FFEFE094F094009534
:106A20001095B094C094D094A194BF0ACF0ADF0A05
:106A3000EF0AFF0A0F0B1F0B0E94343507FC0E9460
:106A40008535CDB7DEB7ECE00C94BB32689401C05D
:106A5000E8948F929F92CF93DF930E943435DF9119
:106A6000CF919F908F90089588249924F401E40198
:106A7000B0E49F93AA279A158B049C04ED05FE05AC
:106A8000CF05D007A10798F4AD2FDC2FCF2FFE2F15
:106A9000E92D982C892E982F872F762F652F542F2C
:106AA000432F322F2227B85031F7BF9127C01B2E1A
:106AB000BF91BB27220F331F441F551F661F771F2F
:106AC000881F991F881C991CEE1FFF1FCC1FDD1FFC
:106AD000AA1FBB1F8A149B04EC05FD05CE05DF052C
:106AE000A007B10748F08A189B08EC09FD09CE09F8
:106AF000DF09A00BB10B21601A94E1F62EF494018A
:106B0000AF01BE01CD01000C089560957095809590
:106B1000909530954095509521953F4F4F4F5F4F41
:106B20006F4F7F4F8F4F9F4F08950F93083090F016
:106B3000982F872F762F652F542F432F322F222700
:106B40000850F4CF220F331F441F551F661F771FB5
:106B5000881F991F0A95B2F70F91089597FB10F8B7
:106B6000169400080F93083098F00850232F342F04
:106B7000452F562F672F782F892F902DF4CF05940E
:106B80009795879577956795579547953795279565
:106B90000A95AAF70F9108952A0D3B1D4C1D5D1D06
:106BA0006E1D7F1D801F911F08952A153B054C0502
:106BB0005D056E057F058007910708950024A7FDF8
:106BC00000942A17300540055005600570058005C2
:106BD00090050895AA1BBB1B51E107C0AA1FBB1F4C
:106BE000A617B70710F0A61BB70B881F991F5A9559
:106BF000A9F780959095BC01CD0108950F931F933F
:106C0000CF93DF938230910510F482E090E0E09121
:106C1000E906F091EA0620E030E0A0E0B0E030972D
:106C200019F1408151810281138148175907C8F039
:106C30008417950769F4109731F012960C93129708
:106C400013961C9327C00093E9061093EA0622C00E
:106C50002115310519F04217530718F49A01BD01A7
:106C6000EF01DF01F801DBCF21153105F9F0281B19
:106C7000390B2430310580F48A819B8161157105BF
:106C800021F0FB019383828304C09093EA068093F2
:106C9000E906FE01329644C0FE01E20FF31F819324
:106CA000919322503109398328833AC02091E70615
:106CB0003091E806232B41F42091890130918A011B
:106CC0003093E8062093E7062091870130918801F0
:106CD0002115310541F42DB73EB740918B015091FC
:106CE0008C01241B350BE091E706F091E806E217D2
:106CF000F307A0F42E1B3F0B2817390778F0AC01DF
:106D00004E5F5F4F2417350748F04E0F5F1F5093BB
:106D1000E8064093E7068193919302C0E0E0F0E03B
:106D2000CF01DF91CF911F910F910895CF93DF9302
:106D3000009709F481C0FC01329713821282A0915E
:106D4000E906B091EA06109781F420813181820F23
:106D5000931F2091E7063091E8062817390751F56F
:106D6000F093E806E093E70667C0ED0120E030E02D
:106D7000CE17DF0740F44A815B819E014115510522
:106D8000F1F0EA01F5CFD383C28340815181840FB2
:106D9000951FC817D90759F488819981840F951FC9
:106DA0000296918380838A819B81938382832115BC
:106DB000310529F4F093EA06E093E9063DC0E901C4
:106DC000FB83EA8349915991C40FD51FEC17FD0746
:106DD00061F480819181840F951F0296E901998366
:106DE0008883828193819B838A83E0E0F0E012961E
:106DF0008D919C911397009719F0FD01DC01F7CF5D
:106E00008D919C9111979D012E5F3F4F820F931F93
:106E10002091E7063091E8062817390769F4309782
:106E200029F41092EA061092E90602C01382128237
:106E3000B093E806A093E706DF91CF910895A0E014
:106E4000B0E0E5E2F7E30C949D32EC01009721F409
:106E5000CB010E94FE35B4C0FC01E60FF71F9C0178
:106E600022503109E217F30708F4A8C0D9010D91A7
:106E70001C91119706171707B0F00530110508F49B
:106E80009BC0C80104978617970708F495C0025065
:106E90001109061B170B019311936D937C93CF017E
:106EA0000E94963689C05B01A01AB10A4C01800E7F
:106EB000911EA091E906B091EA06612C712CE12C9B
:106EC000F12C109709F446C08D919C911197A8154B
:106ED000B905B1F56C0142E0C40ED11CCA14DB0443
:106EE00078F14C018A189B08640142E0C40ED11C61
:106EF0001296BC9012971396AC91B5E0CB16D104C4
:106F000040F0B282A38391828082D9016D937C93F9
:106F100009C00E5F1F4F800F911FF901918380837D
:106F2000EB2DFA2FE114F10431F0D7011396FC9305
:106F3000EE93129741C0F093EA06E093E9063CC055
:106F40006816790608F43C017D0112960D90BC91FB
:106F5000A02DB7CF8091E7069091E8068816990694
:106F6000E1F466167706C8F4809187019091880154
:106F7000009741F48DB79EB740918B0150918C01E1
:106F8000841B950BE817F907C8F4F093E806E09323
:106F9000E706F901718360830FC0CB010E94FE35C3
:106FA0007C01009759F0A801BE010E94EA37CE018A
:106FB0000E949636C70104C0CE0102C080E090E076
:106FC000CDB7DEB7EEE00C94B93281E090E0F894F2
:106FD0000C940338FB01DC0102C001900D9241507A
:106FE0005040D8F70895FB01DC018D910190801984
:106FF0000110D9F3990B0895FB01DC0101900D926A
:107000000020E1F7089510E0C2E7D0E004C0FE01DF
:107010000E945C342196C337D107C9F7F894FFCF9B
:10702000640032001F1115111D1D111F1F111511B4
:107030001515111F1F111D1D1D1D1D1F1F111711BE
:107040001515111F1F1117111D1D111F1F151511CA
:107050001D1D1D1F1F111D111D1D111F70E9D700C2
:10706000F401000005009600C800FA002C015E0142
:107070009001C201F401260258028A02BC02EE020B
:107080002003520384039803A203AC03B603EC9DD0
:107090000200A8FDFFFFB80B000040420F00183DA2
:1070A00087000170E9D7000000EB068000000204B1
:1070B00000030001100302000003020100060004A7
:1070C00000060500200605040000000000A80A15BF
:1070D0000A3F0AF50A700A4E0A620A00000000AE72
:1070E0000B810BDD0B550B790B650B560B0000006C
:1070F00000AE0D150ADD0B140A550053575220201F
:1071000020202020503D30572020202020005357A1
:10711000523D0020503D005720202000FFFFFFFF80
:10712000FFFFFFFF072B363000FFFFFFFFFFFFFFD2
:10713000FF072B353500FFFFFFFFFFFFFFFF072B8A
:10714000353000FFFFFFFFFFFFFFFF072B34350047
:10715000FFFFFFFFFFFFFFFF072B343000FFFFFFA4
:10716000FFFFFFFFFF072B333500FFFFFFFFFFFF90
:10717000FFFF072B333000FFFFFFFFFFFFFFFF077D
:107180002B323500FFFFFFFFFFFFFFFF072B3230E1
:1071900000FFFFFFFFFFFFFFFF072B313500FFFF61
:1071A000FFFFFFFFFFFF072B313000FFFFFFFFFF57
:1071B000FFFFFF072B352000FFFFFFFFFFFFFFFF53
:1071C0000720202000FFFFFFFFFFFFFF06202020F9
:1071D0002000FFFFFFFFFFFF05202020202000FFF1
:1071E000FFFFFFFF0420202020202000FFFFFFFFE3
:1071F000032020202020202000FFFFFF022020204D
:10720000202020202000FFFF0120202020202020FF
:10721000202000FFFF2020202020202020202000F0
:10722000FF2020202020202020202020002020209F
:1072300020202020202020202000436F72722E501A
:107240004C4C2053693533353120200020436F7278
:10725000726563742E2042464F2D3220002020207C
:107260002020434C4B202D203220202020004F6630
:1072700066004F6E2000202020434C4B31203D3EC5
:107280002056464F2020200020203E20434C4B2DEE
:10729000312020202000436F72722E46696C746585
:1072A000722073697A6500487A202020202000200F
:1072B000436F72722E205368696674204357200012
:1072C000436F72722E20535F4C4556454C2D3F0044
:1072D0004C5342004C00555342004641003B0020B5
:1072E0002050494E204130203D2000302042616C2A
:1072F0006C203D204F46462056464F20003320420A
:10730000616C6C3D20302E38206D6B56200036208D
:1073100042616C6C3D2036206D6B56202020003978
:107320002042616C6C3D203530206D6B5620200072
:10733000392B323064423D20353030206D6B562081
:1073400000392B343064423D2035303030206D6BB5
:107350005600392B363064423D2035303030306DA8
:107360006B560031487A20003130487A0035304879
:107370007A0031303048003530304800316B487A7F
:107380000031306B48003130306B004175746F0054
:10739000535342006E616E00696E66006F76660040
:00000001FF
